 ARTLOOK

 Timestamp is 41c7d113 (Mon Dec 20 23:30:27 2004)

 Preferred load address is 00010000

 Start         Length     Name                   Class
 0001:00000000 0002f081H .text                   CODE
 0002:00000000 0000b391H .bss                    DATA
 0003:00000000 00000350H .rdata                  DATA
 0004:00000000 000076c4H .data                   DATA
 0004:000076c8 00000004H .CRT$XCA                DATA
 0004:000076d0 00000004H .CRT$XCZ                DATA
 0004:000076d8 00000004H .CRT$XIA                DATA
 0004:000076dc 00000008H .CRT$XIC                DATA
 0004:000076e8 00000004H .CRT$XIF                DATA
 0004:000076f0 00000004H .CRT$XIG                DATA
 0004:00007700 00000004H .CRT$XIX                DATA
 0004:00007708 00000004H .CRT$XIZ                DATA
 0004:00007710 00000004H .CRT$XPA                DATA
 0004:00007714 00000008H .CRT$XPX                DATA
 0004:00007720 00000004H .CRT$XPZ                DATA
 0004:00007728 00000004H .CRT$XTA                DATA
 0004:00007730 00000004H .CRT$XTZ                DATA
 0005:00000000 00000009H _CONST                  DATA
 0006:00000000 00000014H .idata$2                DATA
 0006:00000014 00000014H .idata$3                DATA
 0006:00000028 00000100H .idata$4                DATA
 0006:00000128 00000100H .idata$5                DATA
 0006:00000228 0000047eH .idata$6                DATA
 0008:00000000 0002b21fH .debug$C                DATA
 0008:0002b220 00001730H .debug$F                DATA
 0008:0002c950 00000000H .debug$G                DATA
 0008:0002c950 00000008H .debug$H                DATA
 0008:0002c958 0000508bH .debug$S                DATA
 0008:000319e3 00004587H .debug$T                DATA

  Address         Publics by Value              Rva+Base   Lib:Object

 0001:fffff000       ___getviewcoord_w          00010000   libf:qcdumb.obj
 0001:fffff000       ___getviewcoord_wxy        00010000   libf:qcdumb.obj
 0001:fffff000       ___getwindowcoord          00010000   libf:qcdumb.obj
 0001:fffff000       ___nfree                   00010000   libf:qcdumb.obj
 0001:fffff000       ___nmalloc                 00010000   libf:qcdumb.obj
 0001:fffff000       ___acrtused                00010000   libf:qcdumb.obj
 0001:fffff000       ___aFldiv                  00010000   libf:qcdumb.obj
 0001:fffff000       ___memmax                  00010000   libf:qcdumb.obj
 0001:fffff000       ___getcurrentposition_w    00010000   libf:qcdumb.obj
 0001:00000000       _main                      00011000 f ARTLOOK.OBJ
 0001:000033fa       _SETLOGICAL@20             000143fa f ARTLOOK.OBJ
 0001:000033fa       _SETLOGICAL                000143fa f ARTLOOK.OBJ
 0001:00003497       _SETREAL@20                00014497 f ARTLOOK.OBJ
 0001:00003497       _SETREAL                   00014497 f ARTLOOK.OBJ
 0001:00003540       _DISPLB@68                 00014540 f DISPLB.OBJ
 0001:00003540       _DISPLB                    00014540 f DISPLB.OBJ
 0001:00006084       _TIMTIK@36                 00017084 f DISPLB.OBJ
 0001:00006084       _TIMTIK                    00017084 f DISPLB.OBJ
 0001:0000659f       _TIMLIN                    0001759f f DISPLB.OBJ
 0001:0000659f       _TIMLIN@36                 0001759f f DISPLB.OBJ
 0001:00006930       _ARTID                     00017930 f INPUT.OBJ
 0001:00006930       _ARTID@16                  00017930 f INPUT.OBJ
 0001:00006ff7       _DECOHEAD                  00017ff7 f INPUT.OBJ
 0001:00006ff7       _DECOHEAD@36               00017ff7 f INPUT.OBJ
 0001:000071b6       _CNVDT@4                   000181b6 f INPUT.OBJ
 0001:000071b6       _CNVDT                     000181b6 f INPUT.OBJ
 0001:00007206       _ARTFREQ@8                 00018206 f INPUT.OBJ
 0001:00007206       _ARTFREQ                   00018206 f INPUT.OBJ
 0001:000076c6       _ARTREAD@28                000186c6 f INPUT.OBJ
 0001:000076c6       _ARTREAD                   000186c6 f INPUT.OBJ
 0001:0000817b       _COPAV                     0001917b f INPUT.OBJ
 0001:0000817b       _COPAV@48                  0001917b f INPUT.OBJ
 0001:00008b70       _NEW_PREPDISP@56           00019b70 f OUTPUT.OBJ
 0001:00008b70       _NEW_PREPDISP              00019b70 f OUTPUT.OBJ
 0001:000091c6       _PREPDISP@52               0001a1c6 f OUTPUT.OBJ
 0001:000091c6       _PREPDISP                  0001a1c6 f OUTPUT.OBJ
 0001:00009ab6       _SAVEART@56                0001aab6 f OUTPUT.OBJ
 0001:00009ab6       _SAVEART                   0001aab6 f OUTPUT.OBJ
 0001:00009fd5       _ARTDUMP                   0001afd5 f OUTPUT.OBJ
 0001:00009fd5       _ARTDUMP@28                0001afd5 f OUTPUT.OBJ
 0001:0000a62b       _SPECMAX@28                0001b62b f OUTPUT.OBJ
 0001:0000a62b       _SPECMAX                   0001b62b f OUTPUT.OBJ
 0001:0000aae0       _CALIBR                    0001bae0 f PROCESS.OBJ
 0001:0000aae0       _CALIBR@52                 0001bae0 f PROCESS.OBJ
 0001:0000aea9       _BACK                      0001bea9 f PROCESS.OBJ
 0001:0000aea9       _BACK@68                   0001bea9 f PROCESS.OBJ
 0001:0000b985       _BACKSUB                   0001c985 f PROCESS.OBJ
 0001:0000b985       _BACKSUB@32                0001c985 f PROCESS.OBJ
 0001:0000bbc4       _BASE@16                   0001cbc4 f PROCESS.OBJ
 0001:0000bbc4       _BASE                      0001cbc4 f PROCESS.OBJ
 0001:0000beb1       _BASE2@20                  0001ceb1 f PROCESS.OBJ
 0001:0000beb1       _BASE2                     0001ceb1 f PROCESS.OBJ
 0001:0000c1d0       _MVCURS                    0001d1d0 f IMAGE:MVCURS.OBJ
 0001:0000c1d0       _MVCURS@44                 0001d1d0 f IMAGE:MVCURS.OBJ
 0001:0000c620       _IMSAVE@8                  0001d620 f IMAGE:IMSAVE.OBJ
 0001:0000c620       _IMSAVE                    0001d620 f IMAGE:IMSAVE.OBJ
 0001:0000cda0       _CNGBUF@20                 0001dda0 f IMAGE:CNGBUF.OBJ
 0001:0000cda0       _CNGBUF                    0001dda0 f IMAGE:CNGBUF.OBJ
 0001:0000cfd0       _PRHEAD@20                 0001dfd0 f UTI:PRHEAD.OBJ
 0001:0000cfd0       _PRHEAD                    0001dfd0 f UTI:PRHEAD.OBJ
 0001:0000d1b0       _XCHGI1                    0001e1b0 f UTI:XCHG.OBJ
 0001:0000d1b0       _XCHGI1@8                  0001e1b0 f UTI:XCHG.OBJ
 0001:0000d1e0       _XCHGI2                    0001e1e0 f UTI:XCHG.OBJ
 0001:0000d1e0       _XCHGI2@8                  0001e1e0 f UTI:XCHG.OBJ
 0001:0000d216       _XCHGI4@8                  0001e216 f UTI:XCHG.OBJ
 0001:0000d216       _XCHGI4                    0001e216 f UTI:XCHG.OBJ
 0001:0000d246       _XCHGR4@8                  0001e246 f UTI:XCHG.OBJ
 0001:0000d246       _XCHGR4                    0001e246 f UTI:XCHG.OBJ
 0001:0000d277       _XCHGR8@8                  0001e277 f UTI:XCHG.OBJ
 0001:0000d277       _XCHGR8                    0001e277 f UTI:XCHG.OBJ
 0001:0000d2c0       _XCHGS                     0001e2c0 f UTI:XCHG.OBJ
 0001:0000d2c0       _XCHGS@20                  0001e2c0 f UTI:XCHG.OBJ
 0001:0000d380       _STAT2                     0001e380 f UTI:STAT2.OBJ
 0001:0000d380       _STAT2@52                  0001e380 f UTI:STAT2.OBJ
 0001:0000d637       _HIST2                     0001e637 f UTI:STAT2.OBJ
 0001:0000d637       _HIST2@52                  0001e637 f UTI:STAT2.OBJ
 0001:0000da40       _VALARGC@16                0001ea40 f UTI:CMDLINE.OBJ
 0001:0000da40       _VALARGC                   0001ea40 f UTI:CMDLINE.OBJ
 0001:0000db77       _VALARGR@8                 0001eb77 f UTI:CMDLINE.OBJ
 0001:0000db77       _VALARGR                   0001eb77 f UTI:CMDLINE.OBJ
 0001:0000dcbe       _VALARGI                   0001ecbe f UTI:CMDLINE.OBJ
 0001:0000dcbe       _VALARGI@8                 0001ecbe f UTI:CMDLINE.OBJ
 0001:0000de04       _COMARG2@8                 0001ee04 f UTI:CMDLINE.OBJ
 0001:0000de04       _COMARG2                   0001ee04 f UTI:CMDLINE.OBJ
 0001:0000dec9       _COMARG                    0001eec9 f UTI:CMDLINE.OBJ
 0001:0000dec9       _COMARG@16                 0001eec9 f UTI:CMDLINE.OBJ
 0001:0000e020       _TIMEWR                    0001f020 f UTI:TIME.OBJ
 0001:0000e020       _TIMEWR@16                 0001f020 f UTI:TIME.OBJ
 0001:0000e14d       _TWR@12                    0001f14d f UTI:TIME.OBJ
 0001:0000e14d       _TWR                       0001f14d f UTI:TIME.OBJ
 0001:0000e19e       _TIM@4                     0001f19e f UTI:TIME.OBJ
 0001:0000e19e       _TIM                       0001f19e f UTI:TIME.OBJ
 0001:0000e227       _DMS@8                     0001f227 f UTI:TIME.OBJ
 0001:0000e227       _DMS                       0001f227 f UTI:TIME.OBJ
 0001:0000e339       _TIMER                     0001f339 f UTI:TIME.OBJ
 0001:0000e339       _TIMER@16                  0001f339 f UTI:TIME.OBJ
 0001:0000e4a0       _FILTSHFT                  0001f4a0 f UTI:FILTSHFT.OBJ
 0001:0000e4a0       _FILTSHFT@32               0001f4a0 f UTI:FILTSHFT.OBJ
 0001:0000f5b0       _FNAM@16                   000205b0 f UTI:FNAM.OBJ
 0001:0000f5b0       _FNAM                      000205b0 f UTI:FNAM.OBJ
 0001:0000f6f0       _KEYGET@12                 000206f0   UTI:KEYBOARD.OBJ
 0001:0000f717       _KEYSTA@16                 00020717   UTI:KEYBOARD.OBJ
 0001:0000f76b       _KEYSHF@4                  0002076b   UTI:KEYBOARD.OBJ
 0001:0000f790       _MOSINI@8                  00020790   UTI:MOUSE.OBJ
 0001:0000f7b6       _MOSVER@16                 000207b6   UTI:MOUSE.OBJ
 0001:0000f7c3       _CURSHO@0                  000207c3   UTI:MOUSE.OBJ
 0001:0000f7d4       _CURHID@0                  000207d4   UTI:MOUSE.OBJ
 0001:0000f7e5       _MOSGET@12                 000207e5   UTI:MOUSE.OBJ
 0001:0000f80a       _MOSSET@8                  0002080a   UTI:MOUSE.OBJ
 0001:0000f817       _MOSPRS@20                 00020817   UTI:MOUSE.OBJ
 0001:0000f824       _MOSRLS@20                 00020824   UTI:MOUSE.OBJ
 0001:0000f831       _MOSXRN@8                  00020831   UTI:MOUSE.OBJ
 0001:0000f83e       _MOSYRN@8                  0002083e   UTI:MOUSE.OBJ
 0001:0000f84b       _MOSDIS@8                  0002084b   UTI:MOUSE.OBJ
 0001:0000f870       _FILEINFO                  00020870 f UTI:FILEINFO.OBJ
 0001:0000f870       _FILEINFO@32               00020870 f UTI:FILEINFO.OBJ
 0001:0000f9c0       _FMIN                      000209c0 f UTI:FMINMAX.OBJ
 0001:0000f9c0       _FMIN@20                   000209c0 f UTI:FMINMAX.OBJ
 0001:0000fe2e       _FMAX                      00020e2e f UTI:FMINMAX.OBJ
 0001:0000fe2e       _FMAX@20                   00020e2e f UTI:FMINMAX.OBJ
 0001:0001029c       _FMINI                     0002129c f UTI:FMINMAX.OBJ
 0001:0001029c       _FMINI@20                  0002129c f UTI:FMINMAX.OBJ
 0001:0001073f       _FMAXI@20                  0002173f f UTI:FMINMAX.OBJ
 0001:0001073f       _FMAXI                     0002173f f UTI:FMINMAX.OBJ
 0001:00010bf0       _POLFIT2                   00021bf0 f UTI:POLFIT2.OBJ
 0001:00010bf0       _POLFIT2@28                00021bf0 f UTI:POLFIT2.OBJ
 0001:00011370       _CONVUC                    00022370 f UTI:CONVUC.OBJ
 0001:00011370       _CONVUC@12                 00022370 f UTI:CONVUC.OBJ
 0001:00011460       _RFFT                      00022460 f UTI:RFFT.OBJ
 0001:00011460       _RFFT@28                   00022460 f UTI:RFFT.OBJ
 0001:00011add       _FFTR                      00022add f UTI:RFFT.OBJ
 0001:00011add       _FFTR@28                   00022add f UTI:RFFT.OBJ
 0001:00011e30       _EXTREM                    00022e30 f UTI:EXTREM.OBJ
 0001:00011e30       _EXTREM@16                 00022e30 f UTI:EXTREM.OBJ
 0001:00011fb0       _DETERM                    00022fb0 f UTI:DETERM.OBJ
 0001:00011fb0       _DETERM@12                 00022fb0 f UTI:DETERM.OBJ
 0001:000123a0       _FFT                       000233a0 f UTI:FFT.OBJ
 0001:000123a0       _FFT@20                    000233a0 f UTI:FFT.OBJ
 0001:00012890       _GAUSSJ@24                 00023890 f UTI:GAUSJ.OBJ
 0001:00012890       _GAUSSJ                    00023890 f UTI:GAUSJ.OBJ
 0001:00013240       _SCREEN                    00024240 f VESA:SCREEN.OBJ
 0001:00013240       _SCREEN@0                  00024240 f VESA:SCREEN.OBJ
 0001:000134e0       _COLREG@4                  000244e0 f VESA:COLREG.OBJ
 0001:000134e0       _COLREG                    000244e0 f VESA:COLREG.OBJ
 0001:00013740       _IMROWX                    00024740 f VESA:IMROWX.OBJ
 0001:00013740       _IMROWX@16                 00024740 f VESA:IMROWX.OBJ
 0001:00013820       _GPRINT@28                 00024820 f VESA:GPRINT.OBJ
 0001:00013820       _GPRINT                    00024820 f VESA:GPRINT.OBJ
 0001:00013c40       _SETMOD@4                  00024c40 f VESA:SETMOD.OBJ
 0001:00013c40       _SETMOD                    00024c40 f VESA:SETMOD.OBJ
 0001:00013c80       _SETCOL                    00024c80 f VESA:SETCOL.OBJ
 0001:00013c80       _SETCOL@12                 00024c80 f VESA:SETCOL.OBJ
 0001:00013d86       _RGB@12                    00024d86 f VESA:SETCOL.OBJ
 0001:00013d86       _RGB                       00024d86 f VESA:SETCOL.OBJ
 0001:00013dc0       _RDROWX                    00024dc0 f VESA:RDROWX.OBJ
 0001:00013dc0       _RDROWX@16                 00024dc0 f VESA:RDROWX.OBJ
 0001:00013ea0       _IMCOLX@16                 00024ea0 f VESA:IMCOLX.OBJ
 0001:00013ea0       _IMCOLX                    00024ea0 f VESA:IMCOLX.OBJ
 0001:00013f80       _RDCOLX@16                 00024f80 f VESA:RDCOLX.OBJ
 0001:00013f80       _RDCOLX                    00024f80 f VESA:RDCOLX.OBJ
 0001:00014060       __FIstrcpy@24              00025060 f libf:intrnchr.obj
 0001:00014100       __FIstraddr@16             00025100 f libf:intrnchr.obj
 0001:00014120       __FIstrcat                 00025120 f libf:intrnchr.obj
 0001:000141c0       __FIpstrcat                000251c0 f libf:intrnchr.obj
 0001:000142d0       __FIdbgstrcpy@32           000252d0 f libf:intrnchr.obj
 0001:00014330       __FIdbgstraddr@20          00025330 f libf:intrnchr.obj
 0001:00014370       __FIdbgstrcat              00025370 f libf:intrnchr.obj
 0001:00014500       __FIdbgpstrcat             00025500 f libf:intrnchr.obj
 0001:00014650       __FIvaxstrcpy@24           00025650 f libf:intrnchr.obj
 0001:000146c0       __FIvaxstrcat              000256c0 f libf:intrnchr.obj
 0001:000147c0       __FIpcleanup@4             000257c0 f libf:intrnchr.obj
 0001:000147d0       __FIclge@16                000257d0 f libf:intrnchr.obj
 0001:00014800       __FIcleq@16                00025800 f libf:intrnchr.obj
 0001:00014830       __FIclne@16                00025830 f libf:intrnchr.obj
 0001:00014860       __FIclgt@16                00025860 f libf:intrnchr.obj
 0001:00014890       __FIclle@16                00025890 f libf:intrnchr.obj
 0001:000148c0       __FIcllt@16                000258c0 f libf:intrnchr.obj
 0001:000148f0       _ccmp@16                   000258f0 f libf:intrnchr.obj
 0001:00014990       __FIindex@20               00025990 f libf:intrnchr.obj
 0001:00014ae0       __FIlentrim@8              00025ae0 f libf:intrnchr.obj
 0001:00014b00       __FIscan@20                00025b00 f libf:intrnchr.obj
 0001:00014c00       __FIverify@20              00025c00 f libf:intrnchr.obj
 0001:00014d00       ___FF_encflt@8             00025d00 f libf:encflt.obj
 0001:00015030       __FFopn                    00026030 f libf:opn.obj
 0001:00015400       __FFalloc                  00026400 f libf:alla.obj
 0001:000154d0       __FFdeall                  000264d0 f libf:alla.obj
 0001:00015560       ___FF_inqputstr@8          00026560 f libf:inq.obj
 0001:000155e0       __FFinq                    000265e0 f libf:inq.obj
 0001:00015ae0       ___FF_decflt@8             00026ae0 f libf:decflt.obj
 0001:00015bd0       ___FF_nrectmo@0            00026bd0 f libf:nrectmo.obj
 0001:00015c40       __FFcls                    00026c40 f libf:cls.obj
 0001:00015d60       ___FF_nrectmi@0            00026d60 f libf:nrectmi.obj
 0001:00015de0       ___FF_nrecfso@0            00026de0 f libf:nrecfso.obj
 0001:00015e30       ___FF_nrecino@0            00026e30 f libf:nrecino.obj
 0001:00015e90       __FFsSTOP                  00026e90 f libf:sstop.obj
 0001:00015ee0       ___FF_ldin@4               00026ee0 f libf:ldin.obj
 0001:00015fc0       ___FF_nrecfsi@0            00026fc0 f libf:nrecfsi.obj
 0001:00016020       ___FF_fmtout@4             00027020 f libf:fmtout.obj
 0001:00016300       ___FF_getchn@0             00027300 f libf:fmtin.obj
 0001:00016410       ___FF_fmtin@4              00027410 f libf:fmtin.obj
 0001:000166b0       ___FF_enclong@12           000276b0 f libf:wr.obj
 0001:00016780       __FFwr                     00027780 f libf:wr.obj
 0001:00016860       ___FF_declong@4            00027860 f libf:rd.obj
 0001:00016900       ___FF_login@0              00027900 f libf:rd.obj
 0001:00016960       __FFrd                     00027960 f libf:rd.obj
 0001:00016a10       __chkstk                   00027a10   libf:chkstk.obj
 0001:00016a70       __setvideomoderows         00027a70   libf:qcsetmod.obj
 0001:00016a8d       __setvideomode             00027a8d   libf:qcsetmod.obj
 0001:00016c02       __settextrows              00027c02   libf:qcsetmod.obj
 0001:00016c72       _$_init_max                00027c72   libf:qcsetmod.obj
 0001:00016ce8       ___FFmathstub              00027ce8   libf:intrin.obj
 0001:00016ce9       __FIfexp                   00027ce9   libf:intrin.obj
 0001:00016d03       __FIcos                    00027d03   libf:intrin.obj
 0001:00016d1d       __FIsin                    00027d1d   libf:intrin.obj
 0001:00016d37       __FItan                    00027d37   libf:intrin.obj
 0001:00016d51       __FIsqrt                   00027d51   libf:intrin.obj
 0001:00016d6b       __FIdprod                  00027d6b   libf:intrin.obj
 0001:00016d6e       __FIlog                    00027d6e   libf:intrin.obj
 0001:00016d88       __FIalog10                 00027d88   libf:intrin.obj
 0001:00016da2       __FIacos                   00027da2   libf:intrin.obj
 0001:00016dbc       __FIcosh                   00027dbc   libf:intrin.obj
 0001:00016dd6       __FIasin                   00027dd6   libf:intrin.obj
 0001:00016df0       __FIsinh                   00027df0   libf:intrin.obj
 0001:00016e0a       __FIatan                   00027e0a   libf:intrin.obj
 0001:00016e24       __FIatan2                  00027e24   libf:intrin.obj
 0001:00016e3e       __FItanh                   00027e3e   libf:intrin.obj
 0001:00016e58       __FIcotan                  00027e58   libf:intrin.obj
 0001:00016e88       __FIexp                    00027e88   libf:intrin.obj
 0001:00016ea2       __FIamod                   00027ea2   libf:intrin.obj
 0001:00016ebc       __FIsign                   00027ebc   libf:intrin.obj
 0001:00016ef0       __FIdim                    00027ef0   libf:intrin.obj
 0001:00016f29       __FIaint                   00027f29   libf:intrin.obj
 0001:00016f29       __FIIaint                  00027f29   libf:intrin.obj
 0001:00016f50       __FIanint                  00027f50   libf:intrin.obj
 0001:00016f50       __FIIanint                 00027f50   libf:intrin.obj
 0001:00016fb9       __FIcdiv                   00027fb9   libf:intrin.obj
 0001:00016fb9       __FIIcdiv                  00027fb9   libf:intrin.obj
 0001:000170b5       __FIcpow                   000280b5   libf:intrin.obj
 0001:000171ab       __FIcabs                   000281ab   libf:intrin.obj
 0001:0001721f       __FIccos                   0002821f   libf:intrin.obj
 0001:00017288       __FIcsin                   00028288   libf:intrin.obj
 0001:000172ef       __FIcexp                   000282ef   libf:intrin.obj
 0001:00017340       __FIclog                   00028340   libf:intrin.obj
 0001:00017394       __FIcsqrt                  00028394   libf:intrin.obj
 0001:00017450       ___FF_hex@0                00028450 f libf:hex.obj
 0001:00017630       __FFuio                    00028630 f libf:uio.obj
 0001:00017900       ___FF_bino@4               00028900 f libf:bino.obj
 0001:00017a60       ___FF_nrecini@0            00028a60 f libf:nrecini.obj
 0001:00017a80       ___FF_bini@4               00028a80 f libf:bini.obj
 0001:00017b40       ___FF_ufdiri@4             00028b40 f libf:ufdiri.obj
 0001:00017c50       _gettok@0                  00028c50 f libf:fmtcr.obj
 0001:00017d40       _putint@4                  00028d40 f libf:fmtcr.obj
 0001:00017d80       _copyint@0                 00028d80 f libf:fmtcr.obj
 0001:00017db0       __FFfmtcr                  00028db0 f libf:fmtcr.obj
 0001:00018410       ___FF_putbint@8            00029410 f libf:tab.obj
 0001:000185e0       ___FF_inrepo@4             000295e0 f libf:tab.obj
 0001:000186f0       ___FF_getnumt@0            000296f0 f libf:tab.obj
 0001:000187b0       ___FF_getchnt@0            000297b0 f libf:tab.obj
 0001:00018850       __FFwr2                    00029850 f libf:wr2.obj
 0001:000188b0       ___FF_ufdiro@4             000298b0 f libf:ufdiro.obj
 0001:00018990       ___FF_ldout@4              00029990 f libf:ldout.obj
 0001:00018a40       ___FF_ufseqi@4             00029a40 f libf:ufseqi.obj
 0001:00018c00       ___FHvexpl@8               00029c00 f libf:helper.obj
 0001:00018c80       ___FHfexpl@8               00029c80 f libf:helper.obj
 0001:00018cc0       ___FHishal@8               00029cc0 f libf:helper.obj
 0001:00018d10       ___FHishll@8               00029d10 f libf:helper.obj
 0001:00018d50       ___FHlink@4                00029d50 f libf:helper.obj
 0001:00018d70       ___FHunlink@0              00029d70 f libf:helper.obj
 0001:00018d80       ___FHbigint@0              00029d80 f libf:helper.obj
 0001:00018da0       ___FHranger@0              00029da0 f libf:helper.obj
 0001:00018dc0       ___FHsranger@0             00029dc0 f libf:helper.obj
 0001:00018de0       ___FHAGOTO@0               00029de0 f libf:helper.obj
 0001:00018e00       ___FHovfl@0                00029e00 f libf:helper.obj
 0001:00018e20       ___FHCASE@0                00029e20 f libf:helper.obj
 0001:00018e40       ___Dollar_debug_unwind     00029e40 f libf:helper.obj
 0001:00018fd0       ___FF_ufseqo@4             00029fd0 f libf:ufseqo.obj
 0001:000191f0       _NARGS@0                   0002a1f0 f libf:args.obj
 0001:00019200       _GETARG@16                 0002a200 f libf:args.obj
 0001:00019290       _GETTIM@16                 0002a290 f libf:timdat.obj
 0001:000192e0       _GETDAT@12                 0002a2e0 f libf:timdat.obj
 0001:00019320       _SETTIM@16                 0002a320 f libf:timdat.obj
 0001:000193f0       _SETDAT@12                 0002a3f0 f libf:timdat.obj
 0001:000194b0       _GETFILEINFOQQ@16          0002a4b0 f libf:files.obj
 0001:00019610       _BadInfo                   0002a610 f libf:files.obj
 0001:00019650       _CopyInfo                  0002a650 f libf:files.obj
 0001:000196a0       _SETFILETIMEQQ@12          0002a6a0 f libf:files.obj
 0001:00019730       _SETFILEACCESSQQ@12        0002a730 f libf:files.obj
 0001:000197b0       _RENAMEFILEQQ@16           0002a7b0 f libf:files.obj
 0001:00019850       _DELFILESQQ@8              0002a850 f libf:files.obj
 0001:00019930       _FINDFILEQQ@24             0002a930 f libf:files.obj
 0001:00019a30       _PACKTIMEQQ@28             0002aa30 f libf:files.obj
 0001:00019ac0       _UNPACKTIMEQQ@28           0002aac0 f libf:files.obj
 0001:00019b70       __FFpPAUSE                 0002ab70 f libf:ppause.obj
 0001:00019bec       __getimage                 0002abec   libf:qcimage.obj
 0001:00019cee       __putimage                 0002acee   libf:qcimage.obj
 0001:00019dd5       __imagesize                0002add5   libf:qcimage.obj
 0001:00019e40       __setcolor                 0002ae40   libf:qcpen.obj
 0001:00019e6f       __getcolor                 0002ae6f   libf:qcpen.obj
 0001:00019e90       __setlinestyle             0002ae90   libf:qcpen.obj
 0001:00019eb9       __getlinestyle             0002aeb9   libf:qcpen.obj
 0001:00019ed2       __remappalette             0002aed2   libf:qcpen.obj
 0001:0001a00e       __remapallpalette          0002b00e   libf:qcpen.obj
 0001:0001a05c       __selectpalette            0002b05c   libf:qcpen.obj
 0001:0001a090       ___FF_puterr@12            0002b090 f libf:puterr.obj
 0001:0001a400       ___FF_error@8              0002b400 f libf:puterr.obj
 0001:0001a590       __arndfstr                 0002b590 f libf:arndfstr.obj
 0001:0001a630       ___FF_getname@4            0002b630 f libf:core.obj
 0001:0001a6a0       ___FF_xerrs@4              0002b6a0 f libf:core.obj
 0001:0001a6e0       __FFend                    0002b6e0 f libf:core.obj
 0001:0001a7f0       __FFinit                   0002b7f0 f libf:core.obj
 0001:0001a940       __FFinit_dll               0002b940 f libf:core.obj
 0001:0001aa80       ___FF_rmblanks@0           0002ba80 f libf:core.obj
 0001:0001aad0       ___FFtk@12                 0002bad0 f libf:core.obj
 0001:0001ac60       ___FFgn@0                  0002bc60 f libf:core.obj
 0001:0001ac70       ___FF_findrec@4            0002bc70 f libf:core.obj
 0001:0001acf0       ___FFpu@4                  0002bcf0 f libf:core.obj
 0001:0001ae60       ___FF_searchunit@4         0002be60 f libf:core.obj
 0001:0001af20       ___FF_searchfile@0         0002bf20 f libf:core.obj
 0001:0001afd0       ___FF_getfip@4             0002bfd0 f libf:core.obj
 0001:0001b040       ___FFio@12                 0002c040 f libf:core.obj
 0001:0001b0c0       ___FF_isdevice@0           0002c0c0 f libf:core.obj
 0001:0001b1b0       ___FF_op@8                 0002c1b0 f libf:core.obj
 0001:0001b740       ___FF_werr@0               0002c740 f libf:core.obj
 0001:0001b780       ___FF_flushbuf@8           0002c780 f libf:core.obj
 0001:0001b8c0       ___FF_chw2r@0              0002c8c0 f libf:core.obj
 0001:0001b940       ___FF_cl@12                0002c940 f libf:core.obj
 0001:0001baf0       ___FF_freefcb@12           0002caf0 f libf:core.obj
 0001:0001bbe0       ___FF_chtmod@0             0002cbe0 f libf:core.obj
 0001:0001bc10       ___FF_oread@8              0002cc10 f libf:core.obj
 0001:0001bd30       ___FF_owrite@4             0002cd30 f libf:core.obj
 0001:0001bd60       ___FF_alloc@4              0002cd60 f libf:core.obj
 0001:0001bd90       ___FF_getfcb@4             0002cd90 f libf:core.obj
 0001:0001be20       ___FF_putds@8              0002ce20 f libf:core.obj
 0001:0001be70       __FFStubFunc@0             0002ce70 f libf:core.obj
 0001:0001be80       _IsWindows                 0002ce80 f libf:core.obj
 0001:0001beb0       _InitNullP                 0002ceb0 f libf:core.obj
 0001:0001bed0       _CheckNullP                0002ced0 f libf:core.obj
 0001:0001bf00       _RError                    0002cf00 f libf:core.obj
 0001:0001bf50       _GetStackSize              0002cf50 f libf:core.obj
 0001:0001bf60       ___FFgi@4                  0002cf60 f libf:gi.obj
 0001:0001bff0       ___FFgm@8                  0002cff0 f libf:getitem.obj
 0001:0001c100       ___FFgs@12                 0002d100 f libf:getitem.obj
 0001:0001c140       ___FF_getitem@4            0002d140 f libf:getitem.obj
 0001:0001c240       ___FF_intin@4              0002d240 f libf:intin.obj
 0001:0001c2b0       ___FF_fillbuf@0            0002d2b0 f libf:fillbuf.obj
 0001:0001c4b0       ___FF_input@0              0002d4b0 f libf:input.obj
 0001:0001c870       ___FF_getred@4             0002d870 f libf:getred.obj
 0001:0001cd30       ___FF_nrecfdo@0            0002dd30   libf:iodec2.obj
 0001:0001cd30       ___FF_nrecfdi@0            0002dd30   libf:iodec2.obj
 0001:0001cd30       _stub0@0                   0002dd30   libf:iodec2.obj
 0001:0001cd33       ___FF_nlin@4               0002dd33   libf:iodec2.obj
 0001:0001cd33       _stub1@4                   0002dd33   libf:iodec2.obj
 0001:0001cd33       ___FF_nlout@4              0002dd33   libf:iodec2.obj
 0001:0001cd3c       _stub2@8                   0002dd3c   libf:iodec2.obj
 0001:0001cd50       ___FF_putbin@8             0002dd50 f libf:putbin.obj
 0001:0001ce20       ___FF_getlong@0            0002de20 f libf:putbin.obj
 0001:0001ce80       ___FF_getnum@0             0002de80 f libf:getnum.obj
 0001:0001d160       ___FF_trunc@0              0002e160 f libf:trunc.obj
 0001:0001d1c0       ___FF_crkrw@0              0002e1c0 f libf:crkrw.obj
 0001:0001d49b       _GetTimeZoneInformation@4  0002e49b f libf:fhack.obj
 0001:0001d539       _OpenProcessToken@12       0002e539 f libf:fhack.obj
 0001:0001d5a3       _AdjustTokenPrivileges@24  0002e5a3 f libf:fhack.obj
 0001:0001d619       _LookupPrivilegeValueA@12  0002e619 f libf:fhack.obj
 0001:0001d683       _GETCHARQQ@8               0002e683 f libf:fhack.obj
 0001:0001d6d8       _PEEKCHARQQ@0              0002e6d8 f libf:fhack.obj
 0001:0001d76c       _GETSTRQQ@8                0002e76c f libf:fhack.obj
 0001:0001d9a0       ___FF_strtol@8             0002e9a0 f libf:fstrtol.obj
 0001:0001db90       ___FF_converchar@4         0002eb90 f libf:fstrtol.obj
 0001:0001dbe0       ___FF_cctl@4               0002ebe0 f libf:cctl.obj
 0001:0001dc50       __grstatus                 0002ec50   libf:qcinit.obj
 0001:0001dc58       _$_SetRows                 0002ec58   libf:qcinit.obj
 0001:0001dc9b       _$_ChkRows                 0002ec9b   libf:qcinit.obj
 0001:0001dd08       _$_FixMaxPage              0002ed08   libf:qcinit.obj
 0001:0001dd47       _$_init_mode               0002ed47   libf:qcinit.obj
 0001:0001dded       ___QCGINIT                 0002eded   libf:qcinit.obj
 0001:0001dee5       ___QCGTERM                 0002eee5   libf:qcinit.obj
 0001:0001df60       _$_qcg_enter               0002ef60   libf:qccore.obj
 0001:0001df97       _$_qcg_exit                0002ef97   libf:qccore.obj
 0001:0001e1af       _$_home_cursor             0002f1af   libf:qccore.obj
 0001:0001e1bf       _$_text_set_cursor         0002f1bf   libf:qccore.obj
 0001:0001e1ee       _$_set_color               0002f1ee   libf:qccore.obj
 0001:0001e21b       _$_set_bk_color            0002f21b   libf:qccore.obj
 0001:0001e2cb       _$_set_text_color          0002f2cb   libf:qccore.obj
 0001:0001e300       _$_set_text_attrib         0002f300   libf:qccore.obj
 0001:0001e348       _$_select_palette          0002f348   libf:qccore.obj
 0001:0001e42a       _$_limit                   0002f42a   libf:qccore.obj
 0001:0001e44b       _$_update_text_cursor      0002f44b   libf:qccore.obj
 0001:0001e47c       _$_unmap_cursor            0002f47c   libf:qccore.obj
 0001:0001e4ab       _$_map_cursor              0002f4ab   libf:qccore.obj
 0001:0001e523       _$_scroll                  0002f523   libf:qccore.obj
 0001:0001e560       _B$ScreenInit              0002f560   libf:llinit.obj
 0001:0001e627       _B$SetAdapter              0002f627   libf:llinit.obj
 0001:0001e8e7       _B$ChkVGA                  0002f8e7   libf:llinit.obj
 0001:0001e90e       _B$ChkMonitor              0002f90e   libf:llinit.obj
 0001:0001e960       _B$SCNIO                   0002f960   libf:llcscn.obj
 0001:0001e96f       _B$GrScreenSize            0002f96f   libf:llcscn.obj
 0001:0001e982       _B$GRMODE                  0002f982   libf:llcscn.obj
 0001:0001e98a       _B$SELVPG                  0002f98a   libf:llcscn.obj
 0001:0001e991       _B$SELAPG                  0002f991   libf:llcscn.obj
 0001:0001e9c3       _B$GETCSRDATA              0002f9c3   libf:llcscn.obj
 0001:0001ea26       _B$OVWCSR                  0002fa26   libf:llcscn.obj
 0001:0001ea2e       _B$OFFCSR                  0002fa2e   libf:llcscn.obj
 0001:0001ea32       _B$CSRDSP                  0002fa32   libf:llcscn.obj
 0001:0001ea91       _B$ErrorReturn             0002fa91   libf:llcscn.obj
 0001:0001eaa0       _B$InitModeData            0002faa0   libf:llcgrp.obj
 0001:0001eb25       _B$MapVWC                  0002fb25   libf:llcgrp.obj
 0001:0001ebd4       _B$OutWord                 0002fbd4   libf:llcgrp.obj
 0001:0001ebdd       _B$ResetEGA                0002fbdd   libf:llcgrp.obj
 0001:0001ec40       _GetDosBlock               0002fc40   libf:dosx.obj
 0001:0001ec59       _FreeDosBlock              0002fc59   libf:dosx.obj
 0001:0001ec73       _B$NearRet                 0002fc73   libf:dosx.obj
 0001:0001ec74       _$_EnsScrSwap              0002fc74   libf:dosx.obj
 0001:0001ec75       _SCNDIR                    0002fc75   libf:dosx.obj
 0001:0001ec76       _B$FarRet                  0002fc76   libf:dosx.obj
 0001:0001ec77       _B$InitSelTable            0002fc77   libf:dosx.obj
 0001:0001ee6d       _B$Screen11                0002fe6d   libf:llvga.obj
 0001:0001eea1       _B$Screen12                0002fea1   libf:llvga.obj
 0001:0001eec3       _B$Screen13                0002fec3   libf:llvga.obj
 0001:0001eedc       _B$Screen102               0002fedc   libf:llvga.obj
 0001:0001ef20       _$_VgaChkRows              0002ff20   libf:llvga.obj
 0001:0001ef8d       _B$VgaSetPages             0002ff8d   libf:llvga.obj
 0001:0001efa0       _B$Vga256PalReset          0002ffa0   libf:llvga.obj
 0001:0001efa7       _B$VgaPalReset             0002ffa7   libf:llvga.obj
 0001:0001eff9       _B$VgaPalPut               0002fff9   libf:llvga.obj
 0001:0001f02a       _B$VgaPalTrans11           0003002a   libf:llvga.obj
 0001:0001f036       _B$VgaPalTrans12           00030036   libf:llvga.obj
 0001:0001f03b       _B$VgaPalTrans13           0003003b   libf:llvga.obj
 0001:0001f06a       _B$SetAttr256              0003006a   libf:llvga.obj
 0001:0001f0a2       _B$VgaLineX256             000300a2   libf:llvga.obj
 0001:0001f15a       _B$VgaLineY256             0003015a   libf:llvga.obj
 0001:0001f222       _B$VgaLineV256             00030222   libf:llvga.obj
 0001:0001f2ca       _B$VgaPutAction_13         000302ca   libf:llvga.obj
 0001:0001f2de       _B$VgaWriteAction256       000302de   libf:llvga.obj
 0001:0001f2ea       _B$VgaNReadL_13            000302ea   libf:llvga.obj
 0001:0001f2f7       _B$VgaNWriteL_13           000302f7   libf:llvga.obj
 0001:0001f327       _B$VgaNSetC_13             00030327   libf:llvga.obj
 0001:0001f379       _B$VgaScanL256             00030379   libf:llvga.obj
 0001:0001f48b       _B$INIT_BKG_MASK13         0003048b   libf:llvga.obj
 0001:0001f656       _b$SimVesaWinFunc          00030656   libf:llvesa.obj
 0001:0001f694       _B$ChkVESA                 00030694   libf:llvesa.obj
 0001:0001f77e       _B$Screen10X               0003077e   libf:llvesa.obj
 0001:0001fa64       _$_VesaInitMaxColor        00030a64   libf:llvesa.obj
 0001:0001fbba       _B$SetVesaWinChk           00030bba   libf:llvesa.obj
 0001:0001fbca       _B$ResetVESA               00030bca   libf:llvesa.obj
 0001:0001fc0f       _B$SetVesaWin              00030c0f   libf:llvesa.obj
 0001:0001fc6a       _B$DecPageC                00030c6a   libf:llvesa.obj
 0001:0001fc7e       _B$IncPageC                00030c7e   libf:llvesa.obj
 0001:0001fce5       _VesaChkDownC              00030ce5   libf:llvesa.obj
 0001:0001fd0e       _VesaDownC                 00030d0e   libf:llvesa.obj
 0001:0001fde7       _B$DecVesaWin              00030de7   libf:llvesa.obj
 0001:0001fdf3       _B$IncVesaWin              00030df3   libf:llvesa.obj
 0001:0001fe08       _VesaNReadL256             00030e08   libf:llvesa.obj
 0001:0001fe30       _VesaNReadL256a            00030e30   libf:llvesa.obj
 0001:0001feb8       _VesaNWriteL256a           00030eb8   libf:llvesa.obj
 0001:00020188       _B$VesaEgaScanLHelper      00031188   libf:llvesa.obj
 0001:000201c7       _B$VesaEgaScanRHelper      000311c7   libf:llvesa.obj
 0001:000202af       _B$Screen4                 000312af   libf:lloga.obj
 0001:00020312       _B$ChkOlivetti             00031312   libf:lloga.obj
 0001:000203a0       __matherr                  000313a0 f libf:matherr.obj
 0001:000207f0       _GetFpArgs                 000317f0 f libf:matherr.obj
 0001:00020870       _SetFpReturn               00031870 f libf:matherr.obj
 0001:00020910       ___FF_mputerr              00031910 f libf:matherr.obj
 0001:00020d10       _FixMathExceptions         00031d10 f libf:matherr.obj
 0001:00020d40       _MathSignal                00031d40 f libf:matherr.obj
 0001:00020d80       _InIntrinsic               00031d80 f libf:matherr.obj
 0001:00020d90       __FFwrite                  00031d90 f libf:ffwrite.obj
 0001:00020e60       ___FF_getu_item@0          00031e60 f libf:ugi.obj
 0001:00020ec0       __FFread                   00031ec0 f libf:ffread.obj
 0001:00020fb0       ___FF_output@0             00031fb0 f libf:output.obj
 0001:000211d0       _FStrToCStr@12             000321d0 f libf:miscproc.obj
 0001:00021240       _CStrToFStr@16             00032240 f libf:miscproc.obj
 0001:000212b0       _GETLASTERRORQQ@0          000322b0 f libf:miscproc.obj
 0001:000212c0       _SETERRORMODEQQ@4          000322c0 f libf:miscproc.obj
 0001:00021300       _GETENVQQ@16               00032300 f libf:miscproc.obj
 0001:00021390       _SETENVQQ@8                00032390 f libf:miscproc.obj
 0001:00021450       _SLEEPQQ@4                 00032450 f libf:miscproc.obj
 0001:00021460       _BEEPQQ@8                  00032460 f libf:miscproc.obj
 0001:00021480       _GETCONFIGQQ@0             00032480 f libf:miscproc.obj
 0001:00021490       _$_coords                  00032490   libf:grputil.obj
 0001:000214bd       _B$INVIEW                  000324bd   libf:grputil.obj
 0001:000214f0       _B$PutGetInit              000324f0   libf:llagrp.obj
 0001:0002156a       _B$NReadC                  0003256a   libf:llagrp.obj
 0001:000215bc       _B$NWriteC                 000325bc   libf:llagrp.obj
 0001:00021619       _B$PaintInit               00032619   libf:llagrp.obj
 0001:00021654       _B$TileMod                 00032654   libf:llagrp.obj
 0001:00021663       _B$StoreC                  00032663   libf:llagrp.obj
 0001:00021679       _B$FetchC                  00032679   libf:llagrp.obj
 0001:00021690       _b$ColorPalette            00032690   libf:llxgasup.obj
 0001:000216a0       _b$EnhPalette              000326a0   libf:llxgasup.obj
 0001:000216ba       _B$EgaPalReset             000326ba   libf:llxgasup.obj
 0001:000216c3       _B$EgaPalResetB            000326c3   libf:llxgasup.obj
 0001:00021703       _B$EgaPalPut               00032703   libf:llxgasup.obj
 0001:0002170c       _B$EgaPalPutB              0003270c   libf:llxgasup.obj
 0001:00021743       _B$EgaPalTrans             00032743   libf:llxgasup.obj
 0001:000217ad       _B$EgaPalSet               000327ad   libf:llxgasup.obj
 0001:00021b70       __FRerror@4                00032b70 f libf:build.obj
 0001:00021cc0       ___FF_dbgmsg@0             00032cc0 f libf:dbgmsg.obj
 0001:0002213a       _B$Screen7                 0003313a   libf:llega.obj
 0001:00022141       _B$Screen8                 00033141   libf:llega.obj
 0001:00022155       _B$Screen9                 00033155   libf:llega.obj
 0001:0002219d       _B$Screen10                0003319d   libf:llega.obj
 0001:000221e9       _B$EgaSetMode              000331e9   libf:llega.obj
 0001:00022720       _B$GRPINI                  00033720   libf:grinit.obj
 0001:00022773       _B$VWINI                   00033773   libf:grinit.obj
 0001:000227a3       _B$VEWINI                  000337a3   libf:grinit.obj
 0001:000227ee       _B$VWMAPC                  000337ee   libf:grinit.obj
 0001:00022831       _B$GRPRST                  00033831   libf:grinit.obj
 0001:00022850       _B$TntInit                 00033850 f libf:tntinit.obj
 0001:00022914       _InitVESA1C                00033914 f libf:tntinit.obj
 0001:0002294c       _SetZeroSeg                0003394c f libf:tntinit.obj
 0001:0002298c       _SetVideoSel               0003398c f libf:tntinit.obj
 0001:00022b3a       _B$Mode0                   00033b3a   libf:lltext.obj
 0001:00022b52       _B$Mode1                   00033b52   libf:lltext.obj
 0001:00022b58       _B$Mode2                   00033b58   libf:lltext.obj
 0001:00022b63       _B$Mode3                   00033b63   libf:lltext.obj
 0001:00022b69       _B$Mode7                   00033b69   libf:lltext.obj
 0001:00022b80       _B$FixTextPage             00033b80   libf:lltext.obj
 0001:00022dee       _B$Mode5                   00033dee   libf:llcga.obj
 0001:00022df4       _B$Mode4                   00033df4   libf:llcga.obj
 0001:00022e4f       _B$Screen2                 00033e4f   libf:llcga.obj
 0001:0002306f       _B$Screen3                 0003406f   libf:llhgc.obj
 0001:00023140       _B$CgaSetAttr              00034140   libf:llcgasup.obj
 0001:0002314b       _B$CgaSetPages             0003414b   libf:llcgasup.obj
 0001:0002315e       _B$MapXYC2                 0003415e   libf:llcgasup.obj
 0001:0002317c       _B$MapXYC2_4               0003417c   libf:llcgasup.obj
 0001:000231a7       _B$CgaReadC                000341a7   libf:llcgasup.obj
 0001:000231ca       _B$CgaSetC                 000341ca   libf:llcgasup.obj
 0001:000231e4       _B$CgaSetPixC              000341e4   libf:llcgasup.obj
 0001:00023201       _B$CgaSetPixFirstC         00034201   libf:llcgasup.obj
 0001:00023208       _B$CgaSetPixLastC          00034208   libf:llcgasup.obj
 0001:00023209       _B$CgaPutAction            00034209   libf:llcgasup.obj
 0001:00023251       _B$CgaNReadL               00034251   libf:llcgasup.obj
 0001:0002326f       _B$CgaNWriteL              0003426f   libf:llcgasup.obj
 0001:000232c8       _B$CgaNSetC                000342c8   libf:llcgasup.obj
 0001:000233bd       _B$CgaSetTile              000343bd   libf:llcgasup.obj
 0001:0002343a       _B$CgaScanL                0003443a   libf:llcgasup.obj
 0001:000234f1       _B$CgaScanR                000344f1   libf:llcgasup.obj
 0001:0002365d       _B$CgaLineX                0003465d   libf:llcgasup.obj
 0001:0002371f       _B$CgaLineY                0003471f   libf:llcgasup.obj
 0001:00023791       _B$CgaLineV                00034791   libf:llcgasup.obj
 0001:00023800       _B$EgaMapXYC_102           00034800   libf:llegasup.obj
 0001:00023816       _B$EgaMapXYC_D             00034816   libf:llegasup.obj
 0001:00023822       _B$EgaMapXYC               00034822   libf:llegasup.obj
 0001:0002387f       _B$EgaLeftC                0003487f   libf:llegasup.obj
 0001:00023888       _B$EgaLeftC_13             00034888   libf:llegasup.obj
 0001:0002388f       _B$EgaChkUpC               0003488f   libf:llegasup.obj
 0001:000238c5       _B$EgaUpC                  000348c5   libf:llegasup.obj
 0001:000238d4       _B$EgaChkDownC             000348d4   libf:llegasup.obj
 0001:0002390a       _B$EgaDownC                0003490a   libf:llegasup.obj
 0001:00023919       _B$EgaSetAttr              00034919   libf:llegasup.obj
 0001:0002392f       _B$EgaReadC                0003492f   libf:llegasup.obj
 0001:0002396f       _B$EgaReadC_F              0003496f   libf:llegasup.obj
 0001:0002397d       _B$EgaReadC_64K            0003497d   libf:llegasup.obj
 0001:00023991       _B$EgaSetC                 00034991   libf:llegasup.obj
 0001:000239cc       _B$EgaSetPixC              000349cc   libf:llegasup.obj
 0001:000239e8       _B$EgaSetPixFirstC         000349e8   libf:llegasup.obj
 0001:00023a04       _B$EgaLineX                00034a04   libf:llegasup.obj
 0001:00023a8a       _B$EgaLineY                00034a8a   libf:llegasup.obj
 0001:00023b08       _B$EgaLineV                00034b08   libf:llegasup.obj
 0001:00023b5d       _B$EgaPutAction_64K        00034b5d   libf:llegasup.obj
 0001:00023b61       _B$EgaPutAction_F          00034b61   libf:llegasup.obj
 0001:00023b65       _B$EgaPutAction            00034b65   libf:llegasup.obj
 0001:00023b9a       _B$EgaNReadL_F             00034b9a   libf:llegasup.obj
 0001:00023b9c       _B$EgaNReadL               00034b9c   libf:llegasup.obj
 0001:00023bdc       _B$EgaNWriteL_F            00034bdc   libf:llegasup.obj
 0001:00023be2       _B$EgaNWriteL              00034be2   libf:llegasup.obj
 0001:00023c8d       _B$EgaNSetC                00034c8d   libf:llegasup.obj
 0001:00023da6       _B$EgaPaintBound           00034da6   libf:llegasup.obj
 0001:00023dab       _B$EgaSetColorBits         00034dab   libf:llegasup.obj
 0001:00023e03       _B$EgaPaintBoundCom        00034e03   libf:llegasup.obj
 0001:00023e59       _B$EgaSetTile              00034e59   libf:llegasup.obj
 0001:00023e7e       _B$EgaScanInit             00034e7e   libf:llegasup.obj
 0001:00023eb0       _B$EgaPAINPX               00034eb0   libf:llegasup.obj
 0001:00023fc7       _B$EgaPIXCNT               00034fc7   libf:llegasup.obj
 0001:00023fd2       _B$EgaSETCMP               00034fd2   libf:llegasup.obj
 0001:00023ff1       _B$EgaCHKBTR               00034ff1   libf:llegasup.obj
 0001:0002400d       _B$EgaCHKBTL               0003500d   libf:llegasup.obj
 0001:0002406e       _B$EgaTILRGT               0003506e   libf:llegasup.obj
 0001:00024170       _B$EgaTILLFT               00035170   libf:llegasup.obj
 0001:000242aa       _B$EgaScanL                000352aa   libf:llegasup.obj
 0001:000243e5       _B$EgaScanR                000353e5   libf:llegasup.obj
 0001:00024520       __clearscreen              00035520   libf:qcclrscn.obj
 0001:000245f0       _B$CgaLeftC2               000355f0   libf:llhgcsup.obj
 0001:000245f6       _B$CgaLeftC1               000355f6   libf:llhgcsup.obj
 0001:00024606       _B$CgaChkUpC               00035606   libf:llhgcsup.obj
 0001:00024625       _B$CgaUpC                  00035625   libf:llhgcsup.obj
 0001:00024641       _B$CgaChkDownC             00035641   libf:llhgcsup.obj
 0001:00024660       _B$CgaDownC                00035660   libf:llhgcsup.obj
 0001:0002467c       _B$CgaPaintBound           0003567c   libf:llhgcsup.obj
 0001:000246c0       _MATHERRQQ@20              000356c0 f libf:mhandler.obj
 0001:000246d0       _B$FPGRINI                 000356d0   libf:grfpinit.obj
 0001:0002472f       _B$WNDINX                  0003572f   libf:grfpinit.obj
 0001:00024778       _B$MAPPX2                  00035778   libf:grfpinit.obj
 0001:0002478a       _B$MAPPY2                  0003578a   libf:grfpinit.obj
 0001:000247c2       _B$ISWNDW                  000357c2   libf:grfpinit.obj
 0001:000247e0       _B$VWFILL                  000357e0   libf:vwclr.obj
 0001:00024816       _B$DOBOXF                  00035816   libf:vwclr.obj
 0001:00024835       _B$SCNFILL                 00035835   libf:vwclr.obj
 0001:00024921       _B$CLIPCK                  00035921   libf:vwclr.obj
 0001:0002499a       _B$XDELT                   0003599a   libf:vwclr.obj
 0001:000249aa       _B$YDELT                   000359aa   libf:vwclr.obj
 0001:000249c0       __outtext                  000359c0   libf:qctext.obj
 0001:00024a4d       __outmem                   00035a4d   libf:qctext.obj
 0001:00024aa7       __inchar                   00035aa7   libf:qctext.obj
 0001:00024b5c       _$_scroll_window           00035b5c   libf:qctext.obj
 0001:00024b9a       _$_fix_text_position       00035b9a   libf:qctext.obj
 0001:00024c40       _B$FastOutStr              00035c40   libf:llscnio.obj
 0001:00024d00       _mainCRTStartup            00035d00 f libc:CRT0.OBJ
 0001:00024e10       __amsg_exit                00035e10 f libc:CRT0.OBJ
 0001:00024e40       __ftol                     00035e40   libc:ftol.obj
 0001:00024e70       __fpmath                   00035e70 f libc:fpinit.obj
 0001:00024e80       __fpclear                  00035e80 f libc:fpinit.obj
 0001:00024e90       __cfltcvt_init             00035e90 f libc:fpinit.obj
 0001:00024ed0       ___setfflag                00035ed0 f libc:fpinit.obj
 0001:00024ee0       _free                      00035ee0 f libc:FREE.OBJ
 0001:00024f40       _realloc                   00035f40 f libc:REALLOC.OBJ
 0001:00025050       __expand                   00036050 f libc:REALLOC.OBJ
 0001:000251f0       _malloc                    000361f0 f libc:MALLOC.OBJ
 0001:000252a0       __heap_split_block         000362a0 f libc:MALLOC.OBJ
 0001:00025300       _memmove                   00036300   libc:MEMMOVE.OBJ
 0001:00025450       _memchr                    00036450   libc:MEMCHR.OBJ
 0001:00025480       __fltout                   00036480 f libc:cfout.obj
 0001:000254f0       ___dtold                   000364f0 f libc:cfout.obj
 0001:000255d0       __cinit                    000365d0 f libc:CRT0DAT.OBJ
 0001:00025600       _exit                      00036600 f libc:CRT0DAT.OBJ
 0001:00025620       __exit                     00036620 f libc:CRT0DAT.OBJ
 0001:00025640       __cexit                    00036640 f libc:CRT0DAT.OBJ
 0001:00025650       __c_exit                   00036650 f libc:CRT0DAT.OBJ
 0001:00025710       __mktemp                   00036710 f libc:MKTEMP.OBJ
 0001:000257e0       __setjmp                   000367e0   libc:SETJMP.OBJ
 0001:0002581f       _longjmp                   0003681f   libc:SETJMP.OBJ
 0001:00025875       _raisex                    00036875   libc:SETJMP.OBJ
 0001:000258b0       __access                   000368b0 f libc:ACCESS.OBJ
 0001:00025900       __fltinf                   00036900 f libc:fltinf.obj
 0001:000259d0       __isatty                   000369d0 f libc:ISATTY.OBJ
 0001:00025a60       __itoa                     00036a60 f libc:XTOA.OBJ
 0001:00025aa0       __ltoa                     00036aa0 f libc:XTOA.OBJ
 0001:00025ad0       __ultoa                    00036ad0 f libc:XTOA.OBJ
 0001:00025af0       _sin                       00036af0   libc:87ctrig.obj
 0001:00025afa       _cos                       00036afa   libc:87ctrig.obj
 0001:00025b01       _tan                       00036b01   libc:87ctrig.obj
 0001:00025b08       __CIsin                    00036b08   libc:87ctrig.obj
 0001:00025b12       __CIcos                    00036b12   libc:87ctrig.obj
 0001:00025b19       __CItan                    00036b19   libc:87ctrig.obj
 0001:00025b20       _sinh                      00036b20   libc:87ctrigh.obj
 0001:00025b2a       _cosh                      00036b2a   libc:87ctrigh.obj
 0001:00025b31       _tanh                      00036b31   libc:87ctrigh.obj
 0001:00025b38       __CIsinh                   00036b38   libc:87ctrigh.obj
 0001:00025b42       __CIcosh                   00036b42   libc:87ctrigh.obj
 0001:00025b49       __CItanh                   00036b49   libc:87ctrigh.obj
 0001:00025b50       _pow                       00036b50   libc:87ctran.obj
 0001:00025b5a       _log                       00036b5a   libc:87ctran.obj
 0001:00025b64       _log10                     00036b64   libc:87ctran.obj
 0001:00025b6b       _exp                       00036b6b   libc:87ctran.obj
 0001:00025b72       __CIpow                    00036b72   libc:87ctran.obj
 0001:00025b7c       __CIlog                    00036b7c   libc:87ctran.obj
 0001:00025b86       __CIlog10                  00036b86   libc:87ctran.obj
 0001:00025b8d       __CIexp                    00036b8d   libc:87ctran.obj
 0001:00025b94       _asin                      00036b94   libc:87ctriga.obj
 0001:00025b9e       _acos                      00036b9e   libc:87ctriga.obj
 0001:00025ba5       _atan                      00036ba5   libc:87ctriga.obj
 0001:00025bac       _atan2                     00036bac   libc:87ctriga.obj
 0001:00025bb6       __CIasin                   00036bb6   libc:87ctriga.obj
 0001:00025bc0       __CIacos                   00036bc0   libc:87ctriga.obj
 0001:00025bc7       __CIatan                   00036bc7   libc:87ctriga.obj
 0001:00025bce       __CIatan2                  00036bce   libc:87ctriga.obj
 0001:00025bd8       _sqrt                      00036bd8   libc:87csqrt.obj
 0001:00025be2       __CIsqrt                   00036be2   libc:87csqrt.obj
 0001:00025bec       _fmod                      00036bec   libc:87fmod.obj
 0001:00025bf6       __CIfmod                   00036bf6   libc:87fmod.obj
 0001:00025c10       __lseek                    00036c10 f libc:LSEEK.OBJ
 0001:00025c90       _strchr                    00036c90   libc:STRCHR.OBJ
 0001:00025cc0       __findfirst                00036cc0 f libc:FINDFILE.OBJ
 0001:00025df0       __findnext                 00036df0 f libc:FINDFILE.OBJ
 0001:00025f20       __findclose                00036f20 f libc:FINDFILE.OBJ
 0001:00025fd0       __utime                    00036fd0 f libc:UTIME.OBJ
 0001:00026010       __futime                   00037010 f libc:UTIME.OBJ
 0001:00026190       _rename                    00037190 f libc:RENAME.OBJ
 0001:000261d0       _remove                    000371d0 f libc:UNLINK.OBJ
 0001:00026200       __unlink                   00037200 f libc:UNLINK.OBJ
 0001:00026210       __searchenv                00037210 f libc:SEARCHEN.OBJ
 0001:00026330       _mktime                    00037330 f libc:MKTIME.OBJ
 0001:00026340       __mkgmtime                 00037340 f libc:MKTIME.OBJ
 0001:000265b0       _localtime                 000375b0 f libc:LOCALTIM.OBJ
 0001:00026760       _system                    00037760 f libc:SYSTEM.OBJ
 0001:00026810       _strncpy                   00037810   libc:STRNCPY.OBJ
 0001:00026840       __onexit                   00037840 f libc:ONEXIT.OBJ
 0001:000268c0       _atexit                    000378c0 f libc:ONEXIT.OBJ
 0001:000268e0       __onexitinit               000378e0 f libc:ONEXIT.OBJ
 0001:00026920       __FF_MSGBANNER             00037920 f libc:CRT0MSG.OBJ
 0001:00026950       __NMSG_WRITE               00037950 f libc:CRT0MSG.OBJ
 0001:000269b0       __GET_RTERRMSG             000379b0 f libc:CRT0MSG.OBJ
 0001:000269f0       __stricmp                  000379f0   libc:STRICMP.OBJ
 0001:000269f0       __strcmpi                  000379f0   libc:STRICMP.OBJ
 0001:00026a40       __fullpath                 00037a40 f libc:FULLPATH.OBJ
 0001:00026d80       __open                     00037d80 f libc:OPEN.OBJ
 0001:00026da0       __sopen                    00037da0 f libc:OPEN.OBJ
 0001:000271a0       __close                    000381a0 f libc:CLOSE.OBJ
 0001:00027240       __write                    00038240 f libc:WRITE.OBJ
 0001:00027470       __toupper                  00038470 f libc:TOUPPER.OBJ
 0001:00027480       _toupper                   00038480 f libc:TOUPPER.OBJ
 0001:000275f0       __chsize                   000385f0 f libc:CHSIZE.OBJ
 0001:00027740       ___tzset                   00038740 f libc:TZSET.OBJ
 0001:00027760       __tzset                    00038760 f libc:TZSET.OBJ
 0001:00027960       __isindst                  00038960 f libc:TZSET.OBJ
 0001:00027a30       _getenv                    00038a30 f libc:GETENV.OBJ
 0001:00027ab0       _memset                    00038ab0   libc:MEMSET.OBJ
 0001:00027b00       __getch                    00038b00 f libc:GETCH.OBJ
 0001:00027be0       __getche                   00038be0 f libc:GETCH.OBJ
 0001:00027c10       __kbhit                    00038c10 f libc:GETCH.OBJ
 0001:00027d10       __ungetch                  00038d10 f libc:GETCH.OBJ
 0001:00027e40       __cputs                    00038e40 f libc:CPUTS.OBJ
 0001:00027e90       __cgets                    00038e90 f libc:CGETS.OBJ
 0001:00027f80       __tolower                  00038f80 f libc:TOLOWER.OBJ
 0001:00027f90       _tolower                   00038f90 f libc:TOLOWER.OBJ
 0001:00028100       _strncmp                   00039100   libc:STRNCMP.OBJ
 0001:00028190       _signal                    00039190 f libc:WINSIG.OBJ
 0001:000282d0       _raise                     000392d0 f libc:WINSIG.OBJ
 0001:00028470       __setmode                  00039470 f libc:SETMODE.OBJ
 0001:00028510       __read                     00039510 f libc:READ.OBJ
 0001:00028730       __strupr                   00039730   libc:STRUPR.OBJ
 0001:00028760       __putenv                   00039760 f libc:PUTENV.OBJ
 0001:00028980       _puts                      00039980 f libc:PUTS.OBJ
 0001:00028a14       __except_handler2          00039a14   libc:EXSUP.OBJ
 0001:00028adf       __global_unwind2           00039adf   libc:EXSUP.OBJ
 0001:00028aff       __unwind_handler           00039aff   libc:EXSUP.OBJ
 0001:00028b25       __local_unwind2            00039b25   libc:EXSUP.OBJ
 0001:00028b8b       __abnormal_termination     00039b8b   libc:EXSUP.OBJ
 0001:00028bc0       __XcptFilter               00039bc0 f libc:WINXFLTR.OBJ
 0001:00028d20       __setenvp                  00039d20 f libc:STDENVP.OBJ
 0001:00028df0       __setargv                  00039df0 f libc:STDARGV.OBJ
 0001:00029010       __ioinit                   0003a010 f libc:IOINIT.OBJ
 0001:00029100       __heap_init                0003a100 f libc:HEAPINIT.OBJ
 0001:00029120       __heap_term                0003a120 f libc:HEAPINIT.OBJ
 0001:00029190       __heap_grow_emptylist      0003a190 f libc:HEAPINIT.OBJ
 0001:000291f0       __setdefaultprecision      0003a1f0 f libc:fp8.obj
 0001:00029210       __forcdecpt                0003a210 f libc:cvt.obj
 0001:00029280       __cropzeros                0003a280 f libc:cvt.obj
 0001:000292e0       __positive                 0003a2e0 f libc:cvt.obj
 0001:00029300       __fassign                  0003a300 f libc:cvt.obj
 0001:00029330       __cftoe                    0003a330 f libc:cvt.obj
 0001:000294a0       __cftof                    0003a4a0 f libc:cvt.obj
 0001:000295d0       __cftog                    0003a5d0 f libc:cvt.obj
 0001:00029690       __cfltcvt                  0003a690 f libc:cvt.obj
 0001:00029730       __heap_abort               0003a730 f libc:HPABORT.OBJ
 0001:00029740       __heap_grow                0003a740 f libc:HEAPGROW.OBJ
 0001:00029840       __heap_grow_region         0003a840 f libc:HEAPGROW.OBJ
 0001:00029900       __heap_free_region         0003a900 f libc:HEAPGROW.OBJ
 0001:00029950       __heap_search              0003a950 f libc:HEAPSRCH.OBJ
 0001:00029a60       _$I10_OUTPUT               0003aa60 f libc:x10fout.obj
 0001:00029e00       __getpid                   0003ae00 f libc:GETPID.OBJ
 0001:00029e10       __dosmaperr                0003ae10 f libc:DOSMAP.OBJ
 0001:00029e90       __ZeroTail                 0003ae90 f libc:intrncvt.obj
 0001:00029f00       __IncMan                   0003af00 f libc:intrncvt.obj
 0001:00029f70       __RoundMan                 0003af70 f libc:intrncvt.obj
 0001:0002a020       __CopyMan                  0003b020 f libc:intrncvt.obj
 0001:0002a040       __FillZeroMan              0003b040 f libc:intrncvt.obj
 0001:0002a060       __IsZeroMan                0003b060 f libc:intrncvt.obj
 0001:0002a080       __ShrMan                   0003b080 f libc:intrncvt.obj
 0001:0002a130       __ld12cvt                  0003b130 f libc:intrncvt.obj
 0001:0002a300       __ld12tod                  0003b300 f libc:intrncvt.obj
 0001:0002a320       __ld12tof                  0003b320 f libc:intrncvt.obj
 0001:0002a340       __ld12told                 0003b340 f libc:intrncvt.obj
 0001:0002a3d0       __atodbl                   0003b3d0 f libc:intrncvt.obj
 0001:0002a410       __atoldbl                  0003b410 f libc:intrncvt.obj
 0001:0002a450       __atoflt                   0003b450 f libc:intrncvt.obj
 0001:0002a490       ___strgtold12              0003b490 f libc:strgtold.obj
 0001:0002abe0       ___STRINGTOLD              0003bbe0 f libc:strgtold.obj
 0001:0002ac30       __fFCOS                    0003bc30   libc:87trig.obj
 0001:0002ac3a       __fFSIN                    0003bc3a   libc:87trig.obj
 0001:0002ac5c       __cintrindisp2             0003bc5c   libc:87cdisp.obj
 0001:0002ac95       __cintrindisp1             0003bc95   libc:87cdisp.obj
 0001:0002acc6       __ctrandisp2               0003bcc6   libc:87cdisp.obj
 0001:0002ae3e       __ctrandisp1               0003be3e   libc:87cdisp.obj
 0001:0002ae65       __fload                    0003be65   libc:87cdisp.obj
 0001:0002aea0       __fFSINH                   0003bea0   libc:87trigh.obj
 0001:0002aef2       __fFCOSH                   0003bef2   libc:87trigh.obj
 0001:0002afad       __fFEXP                    0003bfad   libc:87tran.obj
 0001:0002b004       __rtinfpopse               0003c004   libc:87tran.obj
 0001:0002b006       __rtinfnpopse              0003c006   libc:87tran.obj
 0001:0002b016       __fFLN                     0003c016   libc:87tran.obj
 0001:0002b0cb       __rtinfpop                 0003c0cb   libc:87tran.obj
 0001:0002b0cd       __rtinfnpop                0003c0cd   libc:87tran.obj
 0001:0002b0ea       __ffexpm1                  0003c0ea   libc:87tran.obj
 0001:0002b1b0       __fFATN2                   0003c1b0   libc:87triga.obj
 0001:0002b200       __rtpiby2                  0003c200   libc:87triga.obj
 0001:0002b254       __trandisp1                0003c254   libc:87disp.obj
 0001:0002b2bf       __trandisp2                0003c2bf   libc:87disp.obj
 0001:0002b34f       __rttospopde               0003c34f   libc:87disp.obj
 0001:0002b354       __rttospop                 0003c354   libc:87disp.obj
 0001:0002b356       __rtnospop                 0003c356   libc:87disp.obj
 0001:0002b358       __rttosnpop                0003c358   libc:87disp.obj
 0001:0002b359       __rtnospopde               0003c359   libc:87disp.obj
 0001:0002b360       __rtzeropop                0003c360   libc:87disp.obj
 0001:0002b362       __rtzeronpop               0003c362   libc:87disp.obj
 0001:0002b367       __rtonepop                 0003c367   libc:87disp.obj
 0001:0002b369       __rtonenpop                0003c369   libc:87disp.obj
 0001:0002b36e       __tosnan1                  0003c36e   libc:87disp.obj
 0001:0002b399       __nosnan2                  0003c399   libc:87disp.obj
 0001:0002b39b       __tosnan2                  0003c39b   libc:87disp.obj
 0001:0002b3c6       __nan2                     0003c3c6   libc:87disp.obj
 0001:0002b408       __rtindfpop                0003c408   libc:87disp.obj
 0001:0002b40a       __rtindfnpop               0003c40a   libc:87disp.obj
 0001:0002b41b       __rttosnpopde              0003c41b   libc:87disp.obj
 0001:0002b425       __rtchsifneg               0003c425   libc:87disp.obj
 0001:0002b430       __alloc_osfhnd             0003c430 f libc:OSFINFO.OBJ
 0001:0002b470       __set_osfhnd               0003c470 f libc:OSFINFO.OBJ
 0001:0002b500       __free_osfhnd              0003c500 f libc:OSFINFO.OBJ
 0001:0002b570       __get_osfhandle            0003c570 f libc:OSFINFO.OBJ
 0001:0002b5b0       __open_osfhandle           0003c5b0 f libc:OSFINFO.OBJ
 0001:0002b650       ___gmtotime_t              0003c650 f libc:DTOXTIME.OBJ
 0001:0002b6e0       _gmtime                    0003c6e0 f libc:GMTIME.OBJ
 0001:0002b830       _time                      0003c830 f libc:TIME.OBJ
 0001:0002b890       __getpath                  0003c890 f libc:GETPATH.OBJ
 0001:0002b910       __getcwd                   0003c910 f libc:GETCWD.OBJ
 0001:0002b930       __getdcwd                  0003c930 f libc:GETCWD.OBJ
 0001:0002ba40       __validdrive               0003ca40 f libc:GETCWD.OBJ
 0001:0002ba60       __spawnvpe                 0003ca60 f libc:SPAWNVPE.OBJ
 0001:0002bc60       __spawnve                  0003cc60 f libc:SPAWNVE.OBJ
 0001:0002be90       __msize                    0003ce90 f libc:MSIZE.OBJ
 0001:0002beb0       __getdrive                 0003ceb0 f libc:DRIVE.OBJ
 0001:0002bef0       __chdrive                  0003cef0 f libc:DRIVE.OBJ
 0001:0002bfd0       __isctype                  0003cfd0 f libc:ISCTYPE.OBJ
 0001:0002c090       _atol                      0003d090 f libc:ATOX.OBJ
 0001:0002c140       _atoi                      0003d140 f libc:ATOX.OBJ
 0001:0002c150       __strdup                   0003d150   libc:STRDUP.OBJ
 0001:0002c178       __strnicmp                 0003d178   libc:STRNICMP.OBJ
 0001:0002c1d0       __putch                    0003d1d0 f libc:PUTCH.OBJ
 0001:0002c220       __stbuf                    0003d220 f libc:_SFTBUF.OBJ
 0001:0002c2c0       __ftbuf                    0003d2c0 f libc:_SFTBUF.OBJ
 0001:0002c310       __flsbuf                   0003d310 f libc:_FLSBUF.OBJ
 0001:0002c440       _fwrite                    0003d440 f libc:FWRITE.OBJ
 0001:0002c5b0       __statusfp                 0003d5b0 f libc:ieee87.obj
 0001:0002c5d0       __clearfp                  0003d5d0 f libc:ieee87.obj
 0001:0002c5f0       __control87                0003d5f0 f libc:ieee87.obj
 0001:0002c630       __controlfp                0003d630 f libc:ieee87.obj
 0001:0002c650       __fpreset                  0003d650 f libc:ieee87.obj
 0001:0002c820       __fptrap                   0003d820 f libc:CRT0FP.OBJ
 0001:0002c830       __fptostr                  0003d830 f libc:_FPTOSTR.OBJ
 0001:0002c8c0       __heapadd                  0003d8c0 f libc:HEAPADD.OBJ
 0001:0002c8f0       __heap_addblock            0003d8f0 f libc:HEAPADD.OBJ
 0001:0002cb70       ___addl                    0003db70 f libc:mantold.obj
 0001:0002cba0       ___add_12                  0003dba0 f libc:mantold.obj
 0001:0002cc10       ___shl_12                  0003dc10 f libc:mantold.obj
 0001:0002cc60       ___shr_12                  0003dc60 f libc:mantold.obj
 0001:0002ccb0       ___mtold12                 0003dcb0 f libc:mantold.obj
 0001:0002cda0       ___ld12mul                 0003dda0 f libc:tenpow.obj
 0001:0002d0a0       ___multtenpow12            0003e0a0 f libc:tenpow.obj
 0001:0002d120       __87except                 0003e120 f libc:87except.obj
 0001:0002d250       __powhlp                   0003e250 f libc:powhlp.obj
 0001:0002d4c0       __d_inttype                0003e4c0 f libc:powhlp.obj
 0001:0002d530       __dospawn                  0003e530 f libc:DOSPAWN.OBJ
 0001:0002d780       __cenvarg                  0003e780 f libc:CENVARG.OBJ
 0001:0002daf0       _strrchr                   0003eaf0   libc:STRRCHR.OBJ
 0001:0002db18       _strcat                    0003eb18   libc:STRCAT.OBJ
 0001:0002db1c       _strcpy                    0003eb1c   libc:STRCAT.OBJ
 0001:0002dbb0       _strlen                    0003ebb0   libc:STRLEN.OBJ
 0001:0002dc00       __initcon                  0003ec00 f libc:INITCON.OBJ
 0001:0002dc40       __termcon                  0003ec40 f libc:INITCON.OBJ
 0001:0002dc70       _fflush                    0003ec70 f libc:FFLUSH.OBJ
 0001:0002dcc0       __flush                    0003ecc0 f libc:FFLUSH.OBJ
 0001:0002dd30       __flushall                 0003ed30 f libc:FFLUSH.OBJ
 0001:0002ddb0       __endstdio                 0003edb0 f libc:FFLUSH.OBJ
 0001:0002ddd0       __getbuf                   0003edd0 f libc:_GETBUF.OBJ
 0001:0002de20       __heap_findaddr            0003ee20 f libc:FINDADDR.OBJ
 0001:0002dea0       __handle_qnan1             0003eea0 f libc:fpexcept.obj
 0001:0002df10       __handle_qnan2             0003ef10 f libc:fpexcept.obj
 0001:0002df90       __except1                  0003ef90 f libc:fpexcept.obj
 0001:0002e060       __except2                  0003f060 f libc:fpexcept.obj
 0001:0002e160       __raise_exc                0003f160 f libc:fpexcept.obj
 0001:0002e4f0       __handle_exc               0003f4f0 f libc:fpexcept.obj
 0001:0002e7c0       __umatherr                 0003f7c0 f libc:fpexcept.obj
 0001:0002e870       __set_errno                0003f870 f libc:fpexcept.obj
 0001:0002e8d0       __errcode                  0003f8d0 f libc:fpexcept.obj
 0001:0002e910       __statfp                   0003f910 f libc:fpctrl.obj
 0001:0002e930       __clrfp                    0003f930 f libc:fpctrl.obj
 0001:0002e950       __ctrlfp                   0003f950 f libc:fpctrl.obj
 0001:0002e990       __set_statfp               0003f990 f libc:fpctrl.obj
 0001:0002e9f0       __set_exp                  0003f9f0 f libc:util.obj
 0001:0002ea30       __get_exp                  0003fa30 f libc:util.obj
 0001:0002ea50       __add_exp                  0003fa50 f libc:util.obj
 0001:0002ea80       __set_bexp                 0003fa80 f libc:util.obj
 0001:0002eac0       __sptype                   0003fac0 f libc:util.obj
 0001:0002eb30       __decomp                   0003fb30 f libc:util.obj
 0001:0002ec40       __frnd                     0003fc40 f libc:frnd.obj
 0001:0002ec60       _calloc                    0003fc60 f libc:CALLOC.OBJ
 0001:0002eca0       __commit                   0003fca0 f libc:COMMIT.OBJ
 0001:0002ed00       __fcloseall                0003fd00 f libc:CLOSEALL.OBJ
 0001:0002ed40       _fclose                    0003fd40 f libc:FCLOSE.OBJ
 0001:0002edb0       __freebuf                  0003fdb0 f libc:_FREEBUF.OBJ
 0001:0002edf0       _GetCommandLineA@0         0003fdf0   kernel32:kernel32.def
 0001:0002edf6       _GetLocalTime@4            0003fdf6   kernel32:kernel32.def
 0001:0002edfc       _SetLocalTime@4            0003fdfc   kernel32:kernel32.def
 0001:0002ee02       _GetCurrentProcess@0       0003fe02   kernel32:kernel32.def
 0001:0002ee08       _SetFileAttributesA@8      0003fe08   kernel32:kernel32.def
 0001:0002ee0e       _GetVersion@0              0003fe0e   kernel32:kernel32.def
 0001:0002ee14       _SetHandleCount@4          0003fe14   kernel32:kernel32.def
 0001:0002ee1a       _GetProcAddress@8          0003fe1a   kernel32:kernel32.def
 0001:0002ee20       _LoadLibraryA@4            0003fe20   kernel32:kernel32.def
 0001:0002ee26       _PeekConsoleInputA@16      0003fe26   kernel32:kernel32.def
 0001:0002ee2c       _GetStdHandle@4            0003fe2c   kernel32:kernel32.def
 0001:0002ee32       _SetErrorMode@4            0003fe32   kernel32:kernel32.def
 0001:0002ee38       _Sleep@4                   0003fe38   kernel32:kernel32.def
 0001:0002ee3e       _Beep@8                    0003fe3e   kernel32:kernel32.def
 0001:0002ee44       _GetEnvironmentStrings@0   0003fe44   kernel32:kernel32.def
 0001:0002ee4a       _ExitProcess@4             0003fe4a   kernel32:kernel32.def
 0001:0002ee50       _GetLastError@0            0003fe50   kernel32:kernel32.def
 0001:0002ee56       _GetFileAttributesA@4      0003fe56   kernel32:kernel32.def
 0001:0002ee5c       _SetFilePointer@16         0003fe5c   kernel32:kernel32.def
 0001:0002ee62       _FindFirstFileA@8          0003fe62   kernel32:kernel32.def
 0001:0002ee68       _FindNextFileA@8           0003fe68   kernel32:kernel32.def
 0001:0002ee6e       _FindClose@4               0003fe6e   kernel32:kernel32.def
 0001:0002ee74       _FileTimeToSystemTime@8    0003fe74   kernel32:kernel32.def
 0001:0002ee7a       _SetFileTime@16            0003fe7a   kernel32:kernel32.def
 0001:0002ee80       _SystemTimeToFileTime@8    0003fe80   kernel32:kernel32.def
 0001:0002ee86       _MoveFileA@8               0003fe86   kernel32:kernel32.def
 0001:0002ee8c       _DeleteFileA@4             0003fe8c   kernel32:kernel32.def
 0001:0002ee92       _WriteFile@20              0003fe92   kernel32:kernel32.def
 0001:0002ee98       _CloseHandle@4             0003fe98   kernel32:kernel32.def
 0001:0002ee9e       _GetFileType@4             0003fe9e   kernel32:kernel32.def
 0001:0002eea4       _CreateFileA@28            0003fea4   kernel32:kernel32.def
 0001:0002eeaa       _WideCharToMultiByte@32    0003feaa   kernel32:kernel32.def
 0001:0002eeb0       _LCMapStringW@24           0003feb0   kernel32:kernel32.def
 0001:0002eeb6       _MultiByteToWideChar@24    0003feb6   kernel32:kernel32.def
 0001:0002eebc       _SetEndOfFile@4            0003febc   kernel32:kernel32.def
 0001:0002eec2       _SetConsoleMode@8          0003fec2   kernel32:kernel32.def
 0001:0002eec8       _ReadConsoleInputA@16      0003fec8   kernel32:kernel32.def
 0001:0002eece       _GetConsoleMode@8          0003fece   kernel32:kernel32.def
 0001:0002eed4       _GetNumberOfConsoleInputEvents@8 0003fed4   kernel32:kernel32.def
 0001:0002eeda       _WriteConsoleA@20          0003feda   kernel32:kernel32.def
 0001:0002eee0       _ReadConsoleA@20           0003fee0   kernel32:kernel32.def
 0001:0002eee6       _SetConsoleCtrlHandler@8   0003fee6   kernel32:kernel32.def
 0001:0002eeec       _ReadFile@20               0003feec   kernel32:kernel32.def
 0001:0002eef2       _SetEnvironmentVariableA@8 0003fef2   kernel32:kernel32.def
 0001:0002eef8       _RtlUnwind@16              0003fef8   kernel32:kernel32.def
 0001:0002eefe       _UnhandledExceptionFilter@4 0003fefe   kernel32:kernel32.def
 0001:0002ef04       _GetModuleFileNameA@12     0003ff04   kernel32:kernel32.def
 0001:0002ef0a       _GetStartupInfoA@4         0003ff0a   kernel32:kernel32.def
 0001:0002ef10       _VirtualFree@12            0003ff10   kernel32:kernel32.def
 0001:0002ef16       _VirtualAlloc@16           0003ff16   kernel32:kernel32.def
 0001:0002ef1c       _GetCurrentProcessId@0     0003ff1c   kernel32:kernel32.def
 0001:0002ef22       _SetStdHandle@8            0003ff22   kernel32:kernel32.def
 0001:0002ef28       _GetSystemTime@4           0003ff28   kernel32:kernel32.def
 0001:0002ef2e       _GetCurrentDirectoryA@8    0003ff2e   kernel32:kernel32.def
 0001:0002ef34       _GetFullPathNameA@16       0003ff34   kernel32:kernel32.def
 0001:0002ef3a       _GetLogicalDrives@0        0003ff3a   kernel32:kernel32.def
 0001:0002ef40       _SetCurrentDirectoryA@4    0003ff40   kernel32:kernel32.def
 0001:0002ef46       _GetStringTypeW@16         0003ff46   kernel32:kernel32.def
 0001:0002ef4c       _GetExitCodeProcess@8      0003ff4c   kernel32:kernel32.def
 0001:0002ef52       _WaitForSingleObject@8     0003ff52   kernel32:kernel32.def
 0001:0002ef58       _CreateProcessA@40         0003ff58   kernel32:kernel32.def
 0001:0002ef5e       _RaiseException@16         0003ff5e   kernel32:kernel32.def
 0001:0002ef64       _FlushFileBuffers@4        0003ff64   kernel32:kernel32.def
 0001:0002ef70       __QWINGetDefaultWindow     0003ff70 f console:console.obj
 0001:0002ef85       __QWINGetFileName          0003ff85 f console:console.obj
 0001:0002ef97       __wgopen                   0003ff97 f console:console.obj
 0001:0002efa9       __QWINClose                0003ffa9 f console:console.obj
 0001:0002efbb       __wgsetactive              0003ffbb f console:console.obj
 0001:0002efcd       __wggetactive              0003ffcd f console:console.obj
 0001:0002efdf       __QWINWrite                0003ffdf f console:console.obj
 0001:0002eff1       __QWINRead                 0003fff1 f console:console.obj
 0001:0002f003       _YIELDQQ@0                 00040003 f console:console.obj
 0001:0002f00e       __QWINSetSize              0004000e f console:console.obj
 0001:0002f020       __QWINGetSize              00040020 f console:console.obj
 0001:0002f032       __QWINMsgBox               00040032 f console:console.obj
 0001:0002f044       __QWINRegisterInit         00040044 f console:console.obj
 0001:0002f04f       __QWINRegisterEnd          0004004f f console:console.obj
 0001:0002f05a       __QWINNiceExit             0004005a f console:console.obj
 0001:0002f06c       __QWINSetFocus             0004006c f console:console.obj
 0002:00000000       _ARTEMIS                   00041000   <common>
 0002:00000064       _AUX                       00041064   <common>
 0002:0000006c       _VDU                       0004106c   <common>
 0002:00000084       _fpSetDescriptor           00041084   <common>
 0002:00000088       _fpGetDescriptor           00041088   <common>
 0002:0000008c       _fpRealAlloc               0004108c   <common>
 0002:00000090       _fpRealFree                00041090   <common>
 0002:00000094       _fpRealMap                 00041094   <common>
 0002:00000098       _fpRealCall                00041098   <common>
 0002:0000009c       _fpRealIntr                0004109c   <common>
 0002:000000a0       _VideoSel                  000410a0   <common>
 0002:000000a4       _fpAllocDescriptor         000410a4   <common>
 0002:000000a8       __FFHack                   000410a8   <common>
 0002:000000ac       __FFfirst                  000410ac   <common>
 0002:000000b0       __matherr_flag             000410b0   <common>
 0002:000000b4       __aenvptr                  000410b4   <common>
 0002:000000b8       __bufin                    000410b8   <common>
 0002:000010b8       _matherr_flag              000420b8   <common>
 0002:000010bc       __heap_regions             000420bc   <common>
 0002:000013bc       __heap_descpages           000423bc   <common>
 0002:000013c0       __acmdln                   000423c0   <common>
 0002:000013c4       __pgmptr                   000423c4   <common>
 0002:000013c8       ___onexitend               000423c8   <common>
 0002:000013cc       ___onexitbegin             000423cc   <common>
 0002:0000ae90       __qcg_status               0004be90   libf:qcinit.obj
 0002:0000ae91       _$_arc_info_fValid         0004be91   libf:qcinit.obj
 0002:0000aeb0       _$_current_x               0004beb0   libf:qcdata.obj
 0002:0000aeb2       _$_current_y               0004beb2   libf:qcdata.obj
 0002:0000aeb4       _$_bkg_color               0004beb4   libf:qcdata.obj
 0002:0000aeb8       _$_txt_fg_color            0004beb8   libf:qcdata.obj
 0002:0000aeb9       _$_text_attrib             0004beb9   libf:qcdata.obj
 0002:0000aeba       _$_line_style_mask         0004beba   libf:qcdata.obj
 0002:0000aebc       _$_fill_mask               0004bebc   libf:qcdata.obj
 0002:0000aec4       _$_fill_mask_p             0004bec4   libf:qcdata.obj
 0002:0000aec5       _$_BKG_MASK                0004bec5   libf:qcdata.obj
 0002:0000aed5       _$LINE_DRAWN               0004bed5   libf:qcdata.obj
 0002:0000aed7       _$_text_row                0004bed7   libf:qcdata.obj
 0002:0000aed9       _$_text_column             0004bed9   libf:qcdata.obj
 0002:0000aedb       _$_text_org_row            0004bedb   libf:qcdata.obj
 0002:0000aedd       _$_text_org_col            0004bedd   libf:qcdata.obj
 0002:0000aedf       _$_text_max_row            0004bedf   libf:qcdata.obj
 0002:0000aee1       _$_text_max_col            0004bee1   libf:qcdata.obj
 0002:0000aee3       _$_off_screen              0004bee3   libf:qcdata.obj
 0002:0000aee4       _$_text_wrap_p             0004bee4   libf:qcdata.obj
 0002:0000aee5       _$_cursor_on_screen        0004bee5   libf:qcdata.obj
 0002:0000aee6       _$_old_mode                0004bee6   libf:qcdata.obj
 0002:0000aee8       _b$Buf1                    0004bee8   libf:qcdata.obj
 0002:0000af70       _b$VesaStatus              0004bf70   libf:llinit.obj
 0002:0000af73       _b$VGAmodesH               0004bf73   libf:llinit.obj
 0002:0000af74       _b$WriteMode               0004bf74   libf:llinit.obj
 0002:0000af75       _b$EgaPalSup               0004bf75   libf:llinit.obj
 0002:0000af79       _b$CgaInfo                 0004bf79   libf:llinit.obj
 0002:0000af7a       _b$Adapter                 0004bf7a   libf:llinit.obj
 0002:0000af7b       _b$Monitor                 0004bf7b   libf:llinit.obj
 0002:0000af7c       _b$VideoMem                0004bf7c   libf:llinit.obj
 0002:0000af80       _VideoBaseTableLen         0004bf80   libf:llcgrp.obj
 0002:0000af84       _b$MaskC                   0004bf84   libf:llcgrp.obj
 0002:0000af84       _b$PenC                    0004bf84   libf:llcgrp.obj
 0002:0000af85       _b$AttrC                   0004bf85   libf:llcgrp.obj
 0002:0000af86       _b$OffC                    0004bf86   libf:llcgrp.obj
 0002:0000af86       _b$AddrC                   0004bf86   libf:llcgrp.obj
 0002:0000af8a       _b$SegC                    0004bf8a   libf:llcgrp.obj
 0002:0000af8c       _b$PageC                   0004bf8c   libf:llcgrp.obj
 0002:0000af8e       _b$SaveCp                  0004bf8e   libf:llcgrp.obj
 0002:0000af90       _b$VesaWinFunc             0004bf90   libf:llcgrp.obj
 0002:0000af94       _b$PaintBorder             0004bf94   libf:llcgrp.obj
 0002:0000af95       _b$Tiling                  0004bf95   libf:llcgrp.obj
 0002:0000af96       _b$SaveCa                  0004bf96   libf:llcgrp.obj
 0002:0000af9a       _b$SaveCm                  0004bf9a   libf:llcgrp.obj
 0002:0000af9b       _b$PlaneMask               0004bf9b   libf:llcgrp.obj
 0002:0000af9c       _b$Incr1                   0004bf9c   libf:llcgrp.obj
 0002:0000af9e       _b$Incr2                   0004bf9e   libf:llcgrp.obj
 0002:0000afa0       _b$IncrY                   0004bfa0   libf:llcgrp.obj
 0002:0000afa2       _b$PageL                   0004bfa2   libf:llcgrp.obj
 0002:0000afa4       _B$VTOFST                  0004bfa4   libf:llcgrp.obj
 0002:0000afaa       _B$VBOFST                  0004bfaa   libf:llcgrp.obj
 0002:0000afb0       _B$LEOFST                  0004bfb0   libf:llcgrp.obj
 0002:0000afb6       _B$REOFST                  0004bfb6   libf:llcgrp.obj
 0002:0000afbc       _B$VLOFST                  0004bfbc   libf:llcgrp.obj
 0002:0000afc0       _B$VROFST                  0004bfc0   libf:llcgrp.obj
 0002:0000afc4       _B$VLMASK                  0004bfc4   libf:llcgrp.obj
 0002:0000afc5       _B$VRMASK                  0004bfc5   libf:llcgrp.obj
 0002:0000afc6       _b$BorderColor             0004bfc6   libf:llcgrp.obj
 0002:0000afe2       _B$VesaModeInfo            0004bfe2   libf:llvesa.obj
 0002:0000b022       _b$VesaWin                 0004c022   libf:llvesa.obj
 0002:0000b024       _b$FastVesa                0004c024   libf:llvesa.obj
 0002:0000b052       _regs16                    0004c052   libf:llvesa.obj
 0002:0000b06e       _retVal                    0004c06e   libf:llvesa.obj
 0002:0000b072       _b$VesaRealSeg             0004c072   libf:llvesa.obj
 0002:0000b074       _b$WinFuncPtr              0004c074   libf:llvesa.obj
 0002:0000b090       _B$GRPACX                  0004c090   libf:grdata.obj
 0002:0000b092       _B$GRPACY                  0004c092   libf:grdata.obj
 0002:0000b094       _B$GX_OLD                  0004c094   libf:grdata.obj
 0002:0000b098       _B$GY_OLD                  0004c098   libf:grdata.obj
 0002:0000b09c       _B$GXPOS                   0004c09c   libf:grdata.obj
 0002:0000b09e       _B$GYPOS                   0004c09e   libf:grdata.obj
 0002:0000b0a0       _B$GRFACX                  0004c0a0   libf:grdata.obj
 0002:0000b0a4       _B$GRFACY                  0004c0a4   libf:grdata.obj
 0002:0000b0a8       _B$LINSTL                  0004c0a8   libf:grdata.obj
 0002:0000b0aa       _B$CLINEF                  0004c0aa   libf:grdata.obj
 0002:0000b0ab       _b$ASPECTR                 0004c0ab   libf:grdata.obj
 0002:0000b0ad       _B$CENCNT                  0004c0ad   libf:grdata.obj
 0002:0000b0af       _B$CNPNTS                  0004c0af   libf:grdata.obj
 0002:0000b0b1       _B$CSTCNT                  0004c0b1   libf:grdata.obj
 0002:0000b0b3       _B$CPLOTF                  0004c0b3   libf:grdata.obj
 0002:0000b0b4       _B$COPTFL                  0004c0b4   libf:grdata.obj
 0002:0000b0b5       _B$TILLOC                  0004c0b5   libf:grdata.obj
 0002:0000b0b9       _B$TILFLG                  0004c0b9   libf:grdata.obj
 0002:0000b0ba       _B$TILNDX                  0004c0ba   libf:grdata.obj
 0002:0000b0bb       _B$TILLEN                  0004c0bb   libf:grdata.obj
 0002:0000b0bc       _B$TILHGT                  0004c0bc   libf:grdata.obj
 0002:0000b0bd       _B$TILPTR                  0004c0bd   libf:grdata.obj
 0002:0000b0be       _B$GRPLAN                  0004c0be   libf:grdata.obj
 0002:0000b0bf       _B$WNDWSW                  0004c0bf   libf:grdata.obj
 0002:0000b0c0       _B$WNDWSC                  0004c0c0   libf:grdata.obj
 0002:0000b0c1       _B$VIEWSW                  0004c0c1   libf:grdata.obj
 0002:0000b0d0       _b$EgaPalette              0004c0d0   libf:llxgasup.obj
 0002:0000b150       _B$VXSIZ                   0004c150   libf:grinit.obj
 0002:0000b152       _B$VYSIZ                   0004c152   libf:grinit.obj
 0002:0000b154       _B$VXMIN                   0004c154   libf:grinit.obj
 0002:0000b156       _B$VXMAX                   0004c156   libf:grinit.obj
 0002:0000b158       _B$VYMIN                   0004c158   libf:grinit.obj
 0002:0000b15a       _B$VYMAX                   0004c15a   libf:grinit.obj
 0002:0000b15c       _B$VXOFF                   0004c15c   libf:grinit.obj
 0002:0000b15e       _B$VYOFF                   0004c15e   libf:grinit.obj
 0002:0000b160       _B$VXDIF                   0004c160   libf:grinit.obj
 0002:0000b162       _B$VYDIF                   0004c162   libf:grinit.obj
 0002:0000b170       ___FCclenv                 0004c170   libf:qcdumb.obj
 0002:0000b172       ___asizeC                  0004c172   libf:qcdumb.obj
 0002:0000b173       ___osmode                  0004c173   libf:qcdumb.obj
 0002:0000b174       ___osmajor                 0004c174   libf:qcdumb.obj
 0002:0000b180       _b$PageTable               0004c180   libf:lltext.obj
 0002:0000b1a0       _b$UpSub                   0004c1a0   libf:llcgasup.obj
 0002:0000b1a2       _b$DnSub                   0004c1a2   libf:llcgasup.obj
 0002:0000b1a4       _b$UpDnAdd                 0004c1a4   libf:llcgasup.obj
 0002:0000b1b0       _b$IncrYHi                 0004c1b0   libf:llegasup.obj
 0002:0000b1f0       _B$PXDIF                   0004c1f0   libf:qcfpvars.obj
 0002:0000b1f8       _B$PYDIF                   0004c1f8   libf:qcfpvars.obj
 0002:0000b200       _B$LXDIF                   0004c200   libf:qcfpvars.obj
 0002:0000b208       _B$LYDIF                   0004c208   libf:qcfpvars.obj
 0002:0000b210       _B$WXMIN                   0004c210   libf:qcfpvars.obj
 0002:0000b218       _B$WYMIN                   0004c218   libf:qcfpvars.obj
 0002:0000b220       _B$WXMAX                   0004c220   libf:qcfpvars.obj
 0002:0000b228       _B$WYMAX                   0004c228   libf:qcfpvars.obj
 0003:000002b8       __FFherrout                0004d2b8   libf:core.obj
 0003:000002c0       __FFldintfmt               0004d2c0   libf:core.obj
 0003:000002d8       __FFmaxunits               0004d2d8   libf:unit.obj
 0004:00003a98       __FFopAccess_tab           00051a98   libf:opn.obj
 0004:00003ab8       __FFopBlank_tab            00051ab8   libf:opn.obj
 0004:00003ac8       __FFopStatus_tab           00051ac8   libf:opn.obj
 0004:00003ae8       __FFopForm_tab             00051ae8   libf:opn.obj
 0004:00003b10       __FFopShare_tab            00051b10   libf:opn.obj
 0004:00003b40       __FFopMode_tab             00051b40   libf:opn.obj
 0004:00003b60       __FFtable_tab              00051b60   libf:opn.obj
 0004:00003b88       __FFtypetable              00051b88   libf:opn.obj
 0004:00003ba0       _inqMode_tab               00051ba0   libf:inq.obj
 0004:00003ba4       _inqShare_tab              00051ba4   libf:inq.obj
 0004:00003bb0       _inqAccess_tab             00051bb0   libf:inq.obj
 0004:00003bb8       _inqForm_tab               00051bb8   libf:inq.obj
 0004:00003c60       _inq_s_table               00051c60   libf:inq.obj
 0004:00003d00       __FFclStatus_tab           00051d00   libf:cls.obj
 0004:00003d44       __FFpharlap                00051d44   libf:fortstr.obj
 0004:00003da8       __FFzero                   00051da8   libf:intrin.obj
 0004:00003db0       __FFhalf                   00051db0   libf:intrin.obj
 0004:00003db8       __FFone                    00051db8   libf:intrin.obj
 0004:00003dc0       __FFtwo                    00051dc0   libf:intrin.obj
 0004:00003dc8       __FFten                    00051dc8   libf:intrin.obj
 0004:00003dd0       __FFline                   00051dd0   libf:intrin.obj
 0004:00003e78       _blanks                    00051e78   libf:tab.obj
 0004:000040d0       __FFstktop                 000520d0   libf:core.obj
 0004:000040d4       __FFstkbot                 000520d4   libf:core.obj
 0004:000040d8       __FFstksize                000520d8   libf:core.obj
 0004:000040e0       __FFgd                     000520e0   libf:core.obj
 0004:00004340       __FFTerminate              00052340   libf:core.obj
 0004:00004344       __FFconfig                 00052344   libf:core.obj
 0004:00004348       __FFfn                     00052348   libf:core.obj
 0004:00004450       __FFtype                   00052450   libf:core.obj
 0004:00004460       __FFdatasizes              00052460   libf:core.obj
 0004:00004490       __FFldfltfmt               00052490   libf:core.obj
 0004:000044c0       __FFffsequence             000524c0   libf:core.obj
 0004:000044c8       __FFnewline                000524c8   libf:core.obj
 0004:00004518       __pFFinit                  00052518   libf:core.obj
 0004:00004520       __FFshare_tab              00052520   libf:core.obj
 0004:00004528       __FFmode_tab               00052528   libf:core.obj
 0004:00004530       __FFdevice_info            00052530   libf:core.obj
 0004:00004578       __FFdefault_tab            00052578   libf:core.obj
 0004:00004798       __FFunit_lst               00052798   libf:unit.obj
 0004:000049c8       __FFnextreci_handlers      000529c8   libf:iodec2.obj
 0004:000049d8       __FFnextreco_handlers      000529d8   libf:iodec2.obj
 0004:000049e8       __FFoutput_processors      000529e8   libf:iodec2.obj
 0004:000049f4       __FFinput_processors       000529f4   libf:iodec2.obj
 0004:00004a00       __FFnum_fetchers           00052a00   libf:iodec2.obj
 0004:00004a08       __FFchn_fetchers           00052a08   libf:iodec2.obj
 0004:00004a10       __FFbyte_senders           00052a10   libf:iodec2.obj
 0004:00004a18       __FFunf_rtn_tab            00052a18   libf:iodec2.obj
 0004:00004a30       __FFflt_decoder            00052a30   libf:iodec2.obj
 0004:00004a34       __FFflt_encoder            00052a34   libf:iodec2.obj
 0004:00004a38       __FFhex_handler            00052a38   libf:iodec2.obj
 0004:00004a48       __FFdummy                  00052a48   libf:finit.obj
 0004:00004b28       _ulMaxVals                 00052b28   libf:fstrtol.obj
 0004:00004bc0       ___QCGdummy                00052bc0   libf:fginit.obj
 0004:00004bd0       _b$ScreenX                 00052bd0   libf:qcinit.obj
 0004:00004c31       _$_new_height              00052c31   libf:qcinit.obj
 0004:00004c32       _MyMaxBiosMode             00052c32   libf:qcinit.obj
 0004:00004c40       _b$SavedWin                00052c40   libf:qccore.obj
 0004:00004c50       _scanlinebytes             00052c50   libf:qccore.obj
 0004:00004c60       _$_cursor_enabled          00052c60   libf:qcdata.obj
 0004:00004c61       _B$SEG_ZERO                00052c61   libf:qcdata.obj
 0004:00004c63       _B$SEG_MDPA                00052c63   libf:qcdata.obj
 0004:00004c65       _B$SEG_CGA                 00052c65   libf:qcdata.obj
 0004:00004c67       _B$SEG_EGA                 00052c67   libf:qcdata.obj
 0004:00004c69       _B$SEG_VGA                 00052c69   libf:qcdata.obj
 0004:00004c6b       _B$SEG_MCGA                00052c6b   libf:qcdata.obj
 0004:00004c6d       _B$SEG_HGC                 00052c6d   libf:qcdata.obj
 0004:00004c6f       _B$SEG_OGA                 00052c6f   libf:qcdata.obj
 0004:00004c71       _B$SEG_VESA                00052c71   libf:qcdata.obj
 0004:00004c73       _B$SEG_SuperVGA            00052c73   libf:qcdata.obj
 0004:00004c75       _B$SEG_FUNCTABLE           00052c75   libf:qcdata.obj
 0004:00004c77       _B$SEG_OLI_SYS             00052c77   libf:qcdata.obj
 0004:00004c79       _B$SEG_OLI_ROM             00052c79   libf:qcdata.obj
 0004:00004c7b       _B$SEG_OLI_OPTIONS         00052c7b   libf:qcdata.obj
 0004:00004c7d       _b$BlockSel                00052c7d   libf:qcdata.obj
 0004:00004c7f       _b$BlockRealSeg            00052c7f   libf:qcdata.obj
 0004:00004c81       _b$prev1FVector            00052c81   libf:qcdata.obj
 0004:00004c85       _b$VideoBaseTable          00052c85   libf:qcdata.obj
 0004:00004c8b       _b$SelectorTable           00052c8b   libf:qcdata.obj
 0004:00004c9d       _b$EGASelTable             00052c9d   libf:qcdata.obj
 0004:00004caf       _b$EGAPagAddrs             00052caf   libf:qcdata.obj
 0004:00004cc0       _b$UsrCsrTyp               00052cc0   libf:llinit.obj
 0004:00004cc2       _b$OrgCsrTyp               00052cc2   libf:llinit.obj
 0004:00004cc4       _b$OrgBiosMode             00052cc4   libf:llinit.obj
 0004:00004cc7       _b$orglen                  00052cc7   libf:llinit.obj
 0004:00004cd0       _b$CSRTYP                  00052cd0   libf:llcscn.obj
 0004:00004cd2       _b$CurPages                00052cd2   libf:llcscn.obj
 0004:00004cd2       _b$ActPage                 00052cd2   libf:llcscn.obj
 0004:00004cd3       _b$VisPage                 00052cd3   libf:llcscn.obj
 0004:00004ce0       _b$ScreenMode              00052ce0   libf:llcgrp.obj
 0004:00004ce0       _b$ModeData                00052ce0   libf:llcgrp.obj
 0004:00004ce1       _b$Burst                   00052ce1   libf:llcgrp.obj
 0004:00004ce2       _b$BiosMode                00052ce2   libf:llcgrp.obj
 0004:00004ce4       _b$ScrWidth                00052ce4   libf:llcgrp.obj
 0004:00004ce5       _b$ScrHeight               00052ce5   libf:llcgrp.obj
 0004:00004ce6       _b$HorzRes                 00052ce6   libf:llcgrp.obj
 0004:00004ce8       _b$VertRes                 00052ce8   libf:llcgrp.obj
 0004:00004cea       _b$VideoBase               00052cea   libf:llcgrp.obj
 0004:00004cec       _b$MaxAttr                 00052cec   libf:llcgrp.obj
 0004:00004ced       _b$MaxColor                00052ced   libf:llcgrp.obj
 0004:00004cee       _b$PageSize                00052cee   libf:llcgrp.obj
 0004:00004cef       _b$CurrPSize               00052cef   libf:llcgrp.obj
 0004:00004cf1       _b$MaxPage                 00052cf1   libf:llcgrp.obj
 0004:00004cf2       _b$ForeColor               00052cf2   libf:llcgrp.obj
 0004:00004cf2       _b$FBColors                00052cf2   libf:llcgrp.obj
 0004:00004cf3       _b$EgaWrMd                 00052cf3   libf:llcgrp.obj
 0004:00004cf4       _b$InitPalette             00052cf4   libf:llcgrp.obj
 0004:00004cf8       _b$InitVgaPal              00052cf8   libf:llcgrp.obj
 0004:00004cfc       _b$SetMode                 00052cfc   libf:llcgrp.obj
 0004:00004d00       _b$SetPages                00052d00   libf:llcgrp.obj
 0004:00004d04       _b$PalReset                00052d04   libf:llcgrp.obj
 0004:00004d08       _b$PalPut                  00052d08   libf:llcgrp.obj
 0004:00004d0c       _b$PalTrans                00052d0c   libf:llcgrp.obj
 0004:00004d10       _b$PalSet                  00052d10   libf:llcgrp.obj
 0004:00004d14       _b$BitsPerPixel            00052d14   libf:llcgrp.obj
 0004:00004d15       _b$Planes                  00052d15   libf:llcgrp.obj
 0004:00004d16       _b$BytesPerRow             00052d16   libf:llcgrp.obj
 0004:00004d18       _b$MaskLeft                00052d18   libf:llcgrp.obj
 0004:00004d19       _b$MaskRight               00052d19   libf:llcgrp.obj
 0004:00004d1a       _b$PixelsPerByte           00052d1a   libf:llcgrp.obj
 0004:00004d1c       _b$DivShift                00052d1c   libf:llcgrp.obj
 0004:00004d1d       _b$ModMask                 00052d1d   libf:llcgrp.obj
 0004:00004d1f       _b$Aspect                  00052d1f   libf:llcgrp.obj
 0004:00004d21       _b$AspectInv               00052d21   libf:llcgrp.obj
 0004:00004d23       _b$MapXYC                  00052d23   libf:llcgrp.obj
 0004:00004d27       _b$LeftC                   00052d27   libf:llcgrp.obj
 0004:00004d2b       _b$ChkUpC                  00052d2b   libf:llcgrp.obj
 0004:00004d2f       _b$UpC                     00052d2f   libf:llcgrp.obj
 0004:00004d33       _b$ChkDownC                00052d33   libf:llcgrp.obj
 0004:00004d37       _b$DownC                   00052d37   libf:llcgrp.obj
 0004:00004d3b       _b$SetAttr                 00052d3b   libf:llcgrp.obj
 0004:00004d3f       _b$ReadC                   00052d3f   libf:llcgrp.obj
 0004:00004d43       _b$SetC                    00052d43   libf:llcgrp.obj
 0004:00004d47       _b$SetPixC                 00052d47   libf:llcgrp.obj
 0004:00004d4b       _b$SetPixFirstC            00052d4b   libf:llcgrp.obj
 0004:00004d4f       _b$SetPixLastC             00052d4f   libf:llcgrp.obj
 0004:00004d53       _b$LineX                   00052d53   libf:llcgrp.obj
 0004:00004d57       _b$LineY                   00052d57   libf:llcgrp.obj
 0004:00004d5b       _b$LineV                   00052d5b   libf:llcgrp.obj
 0004:00004d5f       _b$PutAction               00052d5f   libf:llcgrp.obj
 0004:00004d63       _b$NReadL                  00052d63   libf:llcgrp.obj
 0004:00004d67       _b$NWriteL                 00052d67   libf:llcgrp.obj
 0004:00004d6b       _b$NSetC                   00052d6b   libf:llcgrp.obj
 0004:00004d6f       _b$PaintBound              00052d6f   libf:llcgrp.obj
 0004:00004d73       _b$SetTile                 00052d73   libf:llcgrp.obj
 0004:00004d77       _b$ScanL                   00052d77   libf:llcgrp.obj
 0004:00004d7b       _b$ScanR                   00052d7b   libf:llcgrp.obj
 0004:00004d7f       _b$PutVector               00052d7f   libf:llcgrp.obj
 0004:00004db2       _b$VgaPalette              00052db2   libf:llvga.obj
 0004:000050e0       __FFexcept                 000530e0   libf:matherr.obj
 0004:000052a8       __FFerrnum                 000532a8   libf:build.obj
 0004:000052b0       __FFermsg                  000532b0   libf:build.obj
 0004:000053c0       ____aDBswpflg              000533c0   libf:qcdumb.obj
 0004:000053c2       ____aDBswpchk              000533c2   libf:qcdumb.obj
 0004:00005420       _b$Mode2Palette            00053420   libf:llcgasup.obj
 0004:00005422       _b$Mode2VgaPal             00053422   libf:llcgasup.obj
 0004:00005484       __FFDefMathErr             00053484   libf:mhandler.obj
 0004:00005488       __FFerrors                 00053488   libf:errdic.obj
 0004:00005490       __FFer_index               00053490   libf:errdic.obj
 0004:000058d0       __FFer_buffer              000538d0   libf:errdic.obj
 0004:00005dd0       __FFtmap                   00053dd0   libf:errmap.obj
 0004:00005fa4       __aexit_rtn                00053fa4   libc:CRT0.OBJ
 0004:00005fa8       __fltused                  00053fa8   libc:fpinit.obj
 0004:00005fac       __ldused                   00053fac   libc:fpinit.obj
 0004:00005fb0       ___fastflag                00053fb0   libc:fpinit.obj
 0004:00005fb4       __FPinit                   00053fb4   libc:fpinit.obj
 0004:00005fb8       __FPmtinit                 00053fb8   libc:fpinit.obj
 0004:00005fbc       __FPmtterm                 00053fbc   libc:fpinit.obj
 0004:00005fc0       __pnhHeap                  00053fc0   libc:MALLOC.OBJ
 0004:00005fc4       _errno                     00053fc4   libc:CRT0DAT.OBJ
 0004:00005fc8       __doserrno                 00053fc8   libc:CRT0DAT.OBJ
 0004:00005fcc       __umaskval                 00053fcc   libc:CRT0DAT.OBJ
 0004:00005fd0       __osver                    00053fd0   libc:CRT0DAT.OBJ
 0004:00005fd4       __winver                   00053fd4   libc:CRT0DAT.OBJ
 0004:00005fd8       __winmajor                 00053fd8   libc:CRT0DAT.OBJ
 0004:00005fdc       __winminor                 00053fdc   libc:CRT0DAT.OBJ
 0004:00005fe0       ___argc                    00053fe0   libc:CRT0DAT.OBJ
 0004:00005fe4       ___argv                    00053fe4   libc:CRT0DAT.OBJ
 0004:00005fe8       __environ                  00053fe8   libc:CRT0DAT.OBJ
 0004:00005fec       __exitflag                 00053fec   libc:CRT0DAT.OBJ
 0004:00005ff0       __C_Termination_Done       00053ff0   libc:CRT0DAT.OBJ
 0004:00005ff8       __OP_FMODjmptab            00053ff8   libc:87fmod.obj
 0004:00006048       __timezone                 00054048   libc:TIMESET.OBJ
 0004:0000604c       __daylight                 0005404c   libc:TIMESET.OBJ
 0004:00006058       __tzname                   00054058   libc:TIMESET.OBJ
 0004:00006060       ___dnames                  00054060   libc:TIMESET.OBJ
 0004:00006078       ___mnames                  00054078   libc:TIMESET.OBJ
 0004:00006320       __adbgmsg                  00054320   libc:CRT0MSG.OBJ
 0004:00006688       __XcptActTab               00054688   libc:WINXFLTR.OBJ
 0004:00006700       __XcptActTabCount          00054700   libc:WINXFLTR.OBJ
 0004:00006704       __fpecode                  00054704   libc:WINXFLTR.OBJ
 0004:00006708       __pxcptinfoptrs            00054708   libc:WINXFLTR.OBJ
 0004:00006710       __nhandle                  00054710   libc:IOINIT.OBJ
 0004:00006718       __osfile                   00054718   libc:IOINIT.OBJ
 0004:00006758       __osfhnd                   00054758   libc:IOINIT.OBJ
 0004:00006858       __pipech                   00054858   libc:IOINIT.OBJ
 0004:00006898       __heap_desc                00054898   libc:HEAPINIT.OBJ
 0004:000068ac       __heap_resetsize           000548ac   libc:HEAPINIT.OBJ
 0004:000068b0       __amblksiz                 000548b0   libc:HEAPINIT.OBJ
 0004:000068b4       __heap_regionsize          000548b4   libc:HEAPINIT.OBJ
 0004:000068b8       __heap_maxregsize          000548b8   libc:HEAPINIT.OBJ
 0004:000068c0       __cfltcvt_tab              000548c0   libc:CMISCDAT.OBJ
 0004:000069aa       __OP_SINjmptab             000549aa   libc:87trig.obj
 0004:000069ca       __OP_COSjmptab             000549ca   libc:87trig.obj
 0004:000069ea       __OP_TANjmptab             000549ea   libc:87trig.obj
 0004:00006a0c       __OP_SINHjmptab            00054a0c   libc:87trigh.obj
 0004:00006a2c       __OP_COSHjmptab            00054a2c   libc:87trigh.obj
 0004:00006a4c       __OP_TANHjmptab            00054a4c   libc:87trigh.obj
 0004:00006a6c       __infinity                 00054a6c   libc:87tran.obj
 0004:00006a76       __minfinity                00054a76   libc:87tran.obj
 0004:00006a80       __logemax                  00054a80   libc:87tran.obj
 0004:00006ab0       __OP_POWjmptab             00054ab0   libc:87tran.obj
 0004:00006b00       __OP_LOG10jmptab           00054b00   libc:87tran.obj
 0004:00006b20       __OP_LOGjmptab             00054b20   libc:87tran.obj
 0004:00006b40       __OP_EXPjmptab             00054b40   libc:87tran.obj
 0004:00006b60       __OP_ASINjmptab            00054b60   libc:87triga.obj
 0004:00006b80       __OP_ACOSjmptab            00054b80   libc:87triga.obj
 0004:00006ba0       __OP_ATANjmptab            00054ba0   libc:87triga.obj
 0004:00006bc0       __OP_ATAN2jmptab           00054bc0   libc:87triga.obj
 0004:00006c10       __OP_SQRTjmptab            00054c10   libc:87sqrt.obj
 0004:00006c30       __indefinite               00054c30   libc:87disp.obj
 0004:00006c3a       __piby2                    00054c3a   libc:87disp.obj
 0004:00006c4c       __cpower                   00054c4c   libc:87disp.obj
 0004:00006c88       __lpdays                   00054c88   libc:DAYS.OBJ
 0004:00006cc0       __days                     00054cc0   libc:DAYS.OBJ
 0004:00006d34       ___c_onexit                00054d34   libc:CINITONE.OBJ
 0004:00006d38       __pctype                   00054d38   libc:CTYPE.OBJ
 0004:00006d3c       __pwctype                  00054d3c   libc:CTYPE.OBJ
 0004:00006d40       __ctype                    00054d40   libc:CTYPE.OBJ
 0004:00006f44       ___mb_cur_max              00054f44   libc:NLSDATA1.OBJ
 0004:00006f4c       __decimal_point            00054f4c   libc:NLSDATA1.OBJ
 0004:00006f50       __decimal_point_length     00054f50   libc:NLSDATA1.OBJ
 0004:00006f54       __fmode                    00054f54   libc:TXTMODE.OBJ
 0004:00006f58       __lc_handle                00054f58   libc:NLSDATA2.OBJ
 0004:00006f70       __lc_codepage              00054f70   libc:NLSDATA2.OBJ
 0004:00006f74       __coninpfh                 00054f74   libc:CINITCON.OBJ
 0004:00006f78       __confh                    00054f78   libc:CINITCON.OBJ
 0004:00006f80       __stdbuf                   00054f80   libc:_SFTBUF.OBJ
 0004:00006f88       __iob                      00054f88   libc:_FILE.OBJ
 0004:00007208       __lastiob                  00055208   libc:_FILE.OBJ
 0004:0000720c       __p_overlay                0005520c   libc:DOSPAWN.OBJ
 0004:00007220       __cflush                   00055220   libc:CINITSTD.OBJ
 0004:00007228       __pow10pos                 00055228   libc:constpow.obj
 0004:00007388       __pow10neg                 00055388   libc:constpow.obj
 0004:00007698       __d_inf                    00055698   libc:util.obj
 0004:000076a0       __d_ind                    000556a0   libc:util.obj
 0004:000076a8       __d_max                    000556a8   libc:util.obj
 0004:000076b0       __d_min                    000556b0   libc:util.obj
 0004:000076b8       __d_mzero                  000556b8   libc:util.obj
 0004:000076c0       __qw32used                 000556c0   console:console.obj
 0004:000076c8       ___xc_a                    000556c8   libc:crt0init.obj
 0004:000076d0       ___xc_z                    000556d0   libc:crt0init.obj
 0004:000076d8       ___xi_a                    000556d8   libc:crt0init.obj
 0004:00007708       ___xi_z                    00055708   libc:crt0init.obj
 0004:00007710       ___xp_a                    00055710   libc:crt0init.obj
 0004:00007720       ___xp_z                    00055720   libc:crt0init.obj
 0004:00007728       ___xt_a                    00055728   libc:crt0init.obj
 0004:00007730       ___xt_z                    00055730   libc:crt0init.obj
 0005:00000000       _b$FP_1                    00056000   libf:grdata.obj
 0005:00000004       _b$FP_256                  00056004   libf:grdata.obj
 0005:00000008       _B$VIEWSC                  00056008   libf:grdata.obj
 0006:00000000       KERNEL32_IMPORT_DESCRIPTOR 00057000   kernel32:kernel32.def
 0006:00000014       NULL_IMPORT_DESCRIPTOR     00057014   kernel32:kernel32.def
 0006:00000128       __imp__LCMapStringW@24     00057128   kernel32:kernel32.def
 0006:0000012c       __imp__GetLocalTime@4      0005712c   kernel32:kernel32.def
 0006:00000130       __imp__SetLocalTime@4      00057130   kernel32:kernel32.def
 0006:00000134       __imp__GetCurrentProcess@0 00057134   kernel32:kernel32.def
 0006:00000138       __imp__SetFileAttributesA@8 00057138   kernel32:kernel32.def
 0006:0000013c       __imp__GetVersion@0        0005713c   kernel32:kernel32.def
 0006:00000140       __imp__SetHandleCount@4    00057140   kernel32:kernel32.def
 0006:00000144       __imp__GetProcAddress@8    00057144   kernel32:kernel32.def
 0006:00000148       __imp__LoadLibraryA@4      00057148   kernel32:kernel32.def
 0006:0000014c       __imp__PeekConsoleInputA@16 0005714c   kernel32:kernel32.def
 0006:00000150       __imp__GetStdHandle@4      00057150   kernel32:kernel32.def
 0006:00000154       __imp__SetErrorMode@4      00057154   kernel32:kernel32.def
 0006:00000158       __imp__Sleep@4             00057158   kernel32:kernel32.def
 0006:0000015c       __imp__Beep@8              0005715c   kernel32:kernel32.def
 0006:00000160       __imp__GetEnvironmentStrings@0 00057160   kernel32:kernel32.def
 0006:00000164       __imp__ExitProcess@4       00057164   kernel32:kernel32.def
 0006:00000168       __imp__GetLastError@0      00057168   kernel32:kernel32.def
 0006:0000016c       __imp__GetFileAttributesA@4 0005716c   kernel32:kernel32.def
 0006:00000170       __imp__SetFilePointer@16   00057170   kernel32:kernel32.def
 0006:00000174       __imp__FindFirstFileA@8    00057174   kernel32:kernel32.def
 0006:00000178       __imp__FindNextFileA@8     00057178   kernel32:kernel32.def
 0006:0000017c       __imp__FindClose@4         0005717c   kernel32:kernel32.def
 0006:00000180       __imp__FileTimeToSystemTime@8 00057180   kernel32:kernel32.def
 0006:00000184       __imp__SetFileTime@16      00057184   kernel32:kernel32.def
 0006:00000188       __imp__SystemTimeToFileTime@8 00057188   kernel32:kernel32.def
 0006:0000018c       __imp__MoveFileA@8         0005718c   kernel32:kernel32.def
 0006:00000190       __imp__DeleteFileA@4       00057190   kernel32:kernel32.def
 0006:00000194       __imp__WriteFile@20        00057194   kernel32:kernel32.def
 0006:00000198       __imp__CloseHandle@4       00057198   kernel32:kernel32.def
 0006:0000019c       __imp__GetFileType@4       0005719c   kernel32:kernel32.def
 0006:000001a0       __imp__CreateFileA@28      000571a0   kernel32:kernel32.def
 0006:000001a4       __imp__WideCharToMultiByte@32 000571a4   kernel32:kernel32.def
 0006:000001a8       __imp__GetCommandLineA@0   000571a8   kernel32:kernel32.def
 0006:000001ac       __imp__MultiByteToWideChar@24 000571ac   kernel32:kernel32.def
 0006:000001b0       __imp__SetEndOfFile@4      000571b0   kernel32:kernel32.def
 0006:000001b4       __imp__SetConsoleMode@8    000571b4   kernel32:kernel32.def
 0006:000001b8       __imp__ReadConsoleInputA@16 000571b8   kernel32:kernel32.def
 0006:000001bc       __imp__GetConsoleMode@8    000571bc   kernel32:kernel32.def
 0006:000001c0       __imp__GetNumberOfConsoleInputEvents@8 000571c0   kernel32:kernel32.def
 0006:000001c4       __imp__WriteConsoleA@20    000571c4   kernel32:kernel32.def
 0006:000001c8       __imp__ReadConsoleA@20     000571c8   kernel32:kernel32.def
 0006:000001cc       __imp__SetConsoleCtrlHandler@8 000571cc   kernel32:kernel32.def
 0006:000001d0       __imp__ReadFile@20         000571d0   kernel32:kernel32.def
 0006:000001d4       __imp__SetEnvironmentVariableA@8 000571d4   kernel32:kernel32.def
 0006:000001d8       __imp__RtlUnwind@16        000571d8   kernel32:kernel32.def
 0006:000001dc       __imp__UnhandledExceptionFilter@4 000571dc   kernel32:kernel32.def
 0006:000001e0       __imp__GetModuleFileNameA@12 000571e0   kernel32:kernel32.def
 0006:000001e4       __imp__GetStartupInfoA@4   000571e4   kernel32:kernel32.def
 0006:000001e8       __imp__VirtualFree@12      000571e8   kernel32:kernel32.def
 0006:000001ec       __imp__VirtualAlloc@16     000571ec   kernel32:kernel32.def
 0006:000001f0       __imp__GetCurrentProcessId@0 000571f0   kernel32:kernel32.def
 0006:000001f4       __imp__SetStdHandle@8      000571f4   kernel32:kernel32.def
 0006:000001f8       __imp__GetSystemTime@4     000571f8   kernel32:kernel32.def
 0006:000001fc       __imp__GetCurrentDirectoryA@8 000571fc   kernel32:kernel32.def
 0006:00000200       __imp__GetFullPathNameA@16 00057200   kernel32:kernel32.def
 0006:00000204       __imp__GetLogicalDrives@0  00057204   kernel32:kernel32.def
 0006:00000208       __imp__SetCurrentDirectoryA@4 00057208   kernel32:kernel32.def
 0006:0000020c       __imp__GetStringTypeW@16   0005720c   kernel32:kernel32.def
 0006:00000210       __imp__GetExitCodeProcess@8 00057210   kernel32:kernel32.def
 0006:00000214       __imp__WaitForSingleObject@8 00057214   kernel32:kernel32.def
 0006:00000218       __imp__CreateProcessA@40   00057218   kernel32:kernel32.def
 0006:0000021c       __imp__RaiseException@16   0005721c   kernel32:kernel32.def
 0006:00000220       __imp__FlushFileBuffers@4  00057220   kernel32:kernel32.def
 0006:00000224       \177KERNEL32__imp__NULL    00057224   kernel32:kernel32.def

 entry point at        0001:00024d00

 Static symbols

 0001:0001d450       _OnTNT                     0002e450 f libf:fhack.obj
 0001:0002e8a0       __get_fname                0003f8a0 f libc:fpexcept.obj
 0001:0002dd40       _flsall                    0003ed40 f libc:FFLUSH.OBJ
 0001:0002cae0       __before                   0003dae0 f libc:HEAPADD.OBJ
 0001:0002c680       __abstract_cw              0003d680 f libc:ieee87.obj
 0001:0002c730       __hw_cw                    0003d730 f libc:ieee87.obj
 0001:0002c7e0       __abstract_sw              0003d7e0 f libc:ieee87.obj
 0001:0002bbf0       _comexecmd                 0003cbf0 f libc:SPAWNVE.OBJ
 0001:000297b0       __heap_new_region          0003a7b0 f libc:HEAPGROW.OBJ
 0001:00029470       __cftoe_g                  0003a470 f libc:cvt.obj
 0001:000295a0       __cftof_g                  0003a5a0 f libc:cvt.obj
 0001:00029700       __shift                    0003a700 f libc:cvt.obj
 0001:00028ea0       _parse_cmdline             00039ea0 f libc:STDARGV.OBJ
 0001:00028cf0       _xcptlookup                00039cf0 f libc:WINXFLTR.OBJ
 0001:00028920       _findenv                   00039920 f libc:PUTENV.OBJ
 0001:00028140       _ctrlevent_capture@4       00039140 f libc:WINSIG.OBJ
 0001:00028440       _siglookup                 00039440 f libc:WINSIG.OBJ
 0001:00027d40       __getextendedkeycode       00038d40 f libc:GETCH.OBJ
 0001:00026350       __make_time_t              00037350 f libc:MKTIME.OBJ
 0001:00025f50       __timet_from_ft            00036f50 f libc:FINDFILE.OBJ
 0001:000259f0       _xtoa                      000369f0 f libc:XTOA.OBJ
 0001:00025660       _doexit                    00036660 f libc:CRT0DAT.OBJ
 0001:000256e0       __initterm                 000366e0 f libc:CRT0DAT.OBJ
 0001:00025180       __heap_expand_block        00036180 f libc:REALLOC.OBJ

FIXUPS: 25efa ffffff77 5 fffffec1 a a 34 5 5 5 5 1e 9 19 15 29 a 80f 1d
FIXUPS: 26657 5e 12 11 fffffdb6 21 fffffe6c fffffee7 f e c 3f 61 fffffc8a
FIXUPS: 25f6a 2d 20 d 23 c f 23 f 52 73 13 14 f 2a f a32 ffffffe8 fffffff6
FIXUPS: 26b60 fffffff6 ffffffe8 ffffffe8 ffffffe8 ffffffe8 ffffff86 15
FIXUPS: 26ac4 1f fffffe42 30 ffffff61 a 6 ffffffdc fffffff7 ffffffef ffffffde
FIXUPS: 2684c fffffff7 fffffff4 fffffffa ffffffd5 ffffff1f 5f fffffe62
FIXUPS: 265f8 12 9fa 1e 18 6e 1e 67 2e 9 fffffb74 c 9f 10 10 64 9 a3 10
FIXUPS: 26ed3 53 4c 48 fffffc8e 9 11 a ffffff90 fffffff6 fffffff6 fffffff6
FIXUPS: 26bd4 ffffffe8 fffffff6 d14 20 13 fffffe70 1b 3c 37 fffffdd0 24
FIXUPS: 27603 1d 1a fffffcfe 10 1f0 13 28 13 fffffc96 16 5c 1e 61 fffffec9
FIXUPS: 271e4 a 18 ffffff95 e a fffffe2a 1c 1215 d fffffb77 24d 4e c 6
FIXUPS: 28055 a 5 6 2b 3b 20 22 15 e 1a e fffff90c 9e 30 47 47 182 1c fffffbc3
FIXUPS: 2793e 61 fffffea8 1e 12 fe6 19 15 31 2e 47 fffffcc5 39 1a 33 1f
FIXUPS: 286c8 10 9 9 19 12 fffffd89 40 79 28 2e fffffd0b 8d 3c 20 4a fffffdec
FIXUPS: 281e3 d 9 9 101c 34 b4 4b fffffc5d 40 79 28 2e fffffe04 d 17 80
FIXUPS: 28e6f fffffcdd d 1d 2a 31 11 d 5a 18 25 37 1a 12 fffffd97 fffffcca
FIXUPS: 28770 17 cd 12fd ffffffc0 ffffffe2 ffffffd7 ffffffc5 fffffff3 fffffff7
FIXUPS: 29a70 ffffffe9 fffffff2 ffffffe2 ffffff70 13 2d 17 fffffd83 1c
FIXUPS: 297c8 33 3d 33 39 42 6 50 fffffc58 9 36 ab 9 51 fffffb00 1409 3a
FIXUPS: 2a667 15 37 1d 1d 35 fffffad9 ffffff3d 11 32 25 b fffffe70 8d 14
FIXUPS: 29e07 2e 14 10 1c fffffedd 16 2d 11 fffffe22 11e fffffec6 fffffff1
FIXUPS: 29b73 ffffffe8 11b0 34 d 12 d fffffa1d e 52 2b d 8f e e d c 3a
FIXUPS: 2a927 fffffe0c fffffae8 25 d2 f 46 15 32 de 60 28 1f 17 31 3c 153c
FIXUPS: 2bbff 14 fffff328 18 70 12 1a9 1c 21 15 1e 24 e 11 14 18 19 2f
FIXUPS: 2b310 20 4f 6c 12 2e 12 2e 12 fffff984 fffffe5d 1d 72 1230 fffffff3
FIXUPS: 2bf03 fffffff7 ffffffef fffffff9 fffffff5 ffffffda fffffff7 ffffffb6
FIXUPS: 2be59 fffffff1 fffffff0 fffffff3 ffffff0c ffffffea fffffff8 ffffffd9
FIXUPS: 2bcef fffffff1 fffffff2 ffffffe5 fffffff4 ffffffd4 fffffff4 ffffffe4
FIXUPS: 2b699 e8 a8 138 55 da b73 2b fffffd2c fffffff6 fffffeff ffffffe3
FIXUPS: 2c22d fffffff5 fffffff9 ffffffe1 ffffffa2 fffffff7 fffffffa ffffffea
FIXUPS: 2c0c7 ffffffd1 fffffff9 ffffffc9 fffffffb ffffffab fffffffb ffffffe8
FIXUPS: 2bfde ffffffdd ffffffbf fffffffb ffffffea fffffff0 fffffff3 fffffff4
FIXUPS: 2bf31 fffffffb d77 25 81 13 25 24 83 2a d 13 fffffc09 27 15 17
FIXUPS: 2cae8 b6 3f fffffd40 29 56 11 1f 75 fffffdf8 3b fffffc37 13 13
FIXUPS: 2c545 88 9 6 dac 2c 2b 1f fffffe2d 58 51 2c fffffef6 ffffff78 fffffff4
FIXUPS: 2d15a ffffff56 4d 49 ffffff0f 1d fffffe52 17 4c 32 12 f d 10 6
FIXUPS: 2cc0e 27 f d 22 11 1310 175 fffffaa9 15 1a 1a fb 9 e 9 25 47 fffffb56
FIXUPS: 2d901 2a 76 43 29 d 43 3b a2 fffffce9 fffffd9c 21 20 19 27 fffffe93
FIXUPS: 2d4f9 38 fffffe4a 1a36 e fffffe56 1e 19 10 ffffff0c fffffc8a 160
FIXUPS: 2e986 1d fffffc5b cb 7 c d 1f 15 f a 15 1f fffffc90 d4 2b fffffc85
FIXUPS: 2e1e3 12 18 f fffffce2 4f 10dd f 12 30 4c f 4f f 15 14e 158 f 114
FIXUPS: 2f533 29 16a bb 1c 2d 52 d d 1b d fffff583 fffffe9b b 1d 4b 44
FIXUPS: 2ed67 19 fffe6a95 30 30 30 30 ef 77 f0 32 7d 83 7a 1a0ee ffffffa1
FIXUPS: 2fd71 c 1c ffffff7a ffffffb8 9 e ffffff8b fffffe09 173 1a fffff2d3
FIXUPS: 2eef5 5e 22 30 2e 13 fffe60c5 123 12 70 57 c 58 13 2b 11 2b 14
FIXUPS: 153e1 5a 36 5d 6 11 c 24 14 6d 3b 61 c 43 28 41 16 ab 1b 1f 1031
FIXUPS: 16962 95 22 fffff9fc 53 19 c 1b 3c 4a b fffffb33 30 20 20 e 63
FIXUPS: 16161 7e 19 2b 1f 71 1e 16 12 7b 4d fffff98c 15c 121 1321 fffffd0f
FIXUPS: 16f46 2b ffffff20 13 12 10 a fffffea3 16 28 fffffecd 30 9 4b 12
FIXUPS: 16d48 fffffec8 fffffeef 2b 19 12 24 fffffa94 57 5 25 c 2c d bc
FIXUPS: 178e6 48 4e 1b 40 1a fffffd01 aa 1f 56 fffffb37 4f fd 38 25 bc
FIXUPS: 175b9 6 13 1d 13 7a 1a fffff9e4 38 73 25 14 18 53 2b c8 f59 ffffffdf
FIXUPS: 181b8 ffffffea ffffffe0 ffffffec ffffffe4 ffffffe3 ffffffe7 fffffbb3
FIXUPS: 17c28 ffffffae fffffff5 fffffffb fffffffb ffffffe6 ffffffe9 fffffff5
FIXUPS: 17b80 fffffff9 fffffff5 fffffffb fffffffb ffffffe4 fffffff3 ffffffea
FIXUPS: 17a96 ffffffd2 fffffe12 30 16 19 522 ffffffe6 ffffffe6 ffffffe6
FIXUPS: 17d93 ffffffe6 ffffffe3 ffffffe6 ffffffe6 ffffffe6 ffffffe6 745
FIXUPS: 18401 ffffffdb ffffffc5 ffffffea ffffffe1 ffffffe7 fffffff4 fffffff0
FIXUPS: 18322 ffffffee ffffffee fffffff8 fffffff0 ffffffd9 ffffffdc fffffff4
FIXUPS: 1827f ffffffd9 ffffffda fffffff4 828 fffffc38 94 11 25 1f 23 25
FIXUPS: 18813 1c 24 30 35 fffffd31 fffffad9 ffffffea ffffffe2 ffffff38
FIXUPS: 17fb0 ffffffad ffffffc2 ffffffd8 fffffff0 ffffffdc ffffffea ffffffe6
FIXUPS: 17e7f ffffffe8 fffffff8 ffffffea ffffffe6 ffffffe6 11e2 16 39 12
FIXUPS: 190d7 1a 10 2f 11 16 5a 29 18 d 10 29 5 1a 46 fffff8bd 89 10 3c
FIXUPS: 18a8b 6f 29 fffffdf9 86 2b 3a 1b 20 e79 71 45 ffffff12 fffffbd6
FIXUPS: 194e9 37 2d 31 af 2f 22 1b 69 96 5d fffff4eb a1 1a d 3b 10 32 2c
FIXUPS: 18e56 83 42 a 1c 30 1c 37 1485 32 25 fffffb8a 83 104 14 d 10 fffffa8f
FIXUPS: 19d8f 20 20 20 20 20 36 74 19 22 12 23 1c 3b fffffac4 39 77 43
FIXUPS: 19bdb 15 fffffde4 14 e42 d 3a 1c 14 1c 17 1d 13 12 38 1a 25 24
FIXUPS: 1a9be d 4e 81 3d fffff7c3 4f 43 c 6 18 23 42 25 1c c 6 18 89e fffffff1
FIXUPS: 1aca9 ffffff7d ffffffdc fffffff1 ffffff84 19 c f 27 fffff915 12
FIXUPS: 1a529 2d 1e 21 15 19 f f b6 2e 3a f 57 1b 1a 2a 14 25 1e 8b0 1a
FIXUPS: 1b113 f 22 39 1f 11 12 8 12 3e 7b 135 8 e a 62 c2 5e 19 fffffaf1
FIXUPS: 1b063 ffffffb3 fffffec5 ffffff80 ffffff5a ffffffeb fffffff4 ffffffef
FIXUPS: 1ad15 ffffffe2 1d5d 1d 42 46 c 9 23 d d d d d 95 26 2e 4c 3c 20
FIXUPS: 1cd4a 1d 12 1c 10 13 73 2f 6 88 2a 24 e ffffe17f 12c2 18 90 c2
FIXUPS: 1c4f8 15 16 18 53 33 32 52 2c 15 3a 68 2a 1c 6f 12 c 16 67 38 4b
FIXUPS: 1c91f 7b 29 3c 1c 6 13 fffff3a1 a 14 1d 14 11 a f c e2 19 24 18
FIXUPS: 1bfa3 3d 45 4a 2e c 6c 1a b3 18 16 24 66 2d 41 3e a 16 19 fffff539
FIXUPS: 1b8c2 10 e 11 3f 13 23 a 3f 2a 10 1f a 10 e 11 159 17 18 17 19
FIXUPS: 1bc10 19 3d 5 51 19 66 42 17 32 1a4e 16 fffffb22 b 25 3d 24 75
FIXUPS: 1d466 fffffe3a fffffe6c 23 79 b 3c 2f e ffffe421 30 3d 10 41 53
FIXUPS: 1b770 66 11 c 23 a 3f 2a 10 28f2 c 17 fffffd09 92 83 fffffdbc fffffbc6
FIXUPS: 1db77 2c d d d d d d d d d d d d fffff8cf 32 37 ce b 16 fe 6 d
FIXUPS: 1d795 e42 4c 12 18 40 1f 36 16 18 69 2b d 25 24 24 16 16 16 90
FIXUPS: 1e22f 13 52 8 20 19 32 26 21 23 34 1c 16 aa0 ffffffc0 fffffff2
FIXUPS: 1ee22 ffffffd9 fffffffb fffffffb ffffffb1 ffffffe7 ffffffc6 fffffff9
FIXUPS: 1ed42 ffffffc7 ffffffbb ffffffc5 ffffffae fffffe2e 147 e e fffff892
FIXUPS: 1e4a5 12 18 29 d 10 2e 12 18 40 12 1b7f fffffff9 ffffffbe fffffff9
FIXUPS: 1fc7d fffffe89 ffffff80 fffffe6d ffffff0d ffffffda ffffff25 ffffff52
FIXUPS: 1f64a ffffffca ffffffa2 39f fffff914 fffffeb1 fffffed1 ffffffe6
FIXUPS: 1ef61 5ec ffffffef fffffffb fffffff9 ffffff48 fffffffb fffffa65
FIXUPS: 1eec2 ffffffe8 ffffffe5 fffffff5 1c5f ffffff28 ffffff29 745 fffffee6
FIXUPS: 20de3 ffffffbd ffffffc2 485 fffffffb ffffffc0 fffffffb ffffff6a
FIXUPS: 1fff3 ffffffea ffffffe4 ffffffc7 ffffffde ffffff57 513 fffffff9
FIXUPS: 2037d ffffff38 fffffff9 ffffffd9 fffffff9 ffffffde fffffff9 ffffffae
FIXUPS: 201fe ffffffb6 fffffff9 1df1 fffffee7 14 18 ffffff02 24 1f 23 15
FIXUPS: 21e46 fffff5fa 3c 8b 54 1d 337 d 126 34f 13 1c 16 fffff598 ffffffdb
FIXUPS: 212c3 fffff58d ffffff61 ffffffc3 ffffff2e 45b fffffff9 fffffffb
FIXUPS: 23550 fffff7cb 1d 26 14 fffff944 fffffffb fffffb42 15 c4 9 e 9
FIXUPS: 22315 1b d 40 28 31 17 2b 40 1f fffffbf2 1e 10d fffffd55 9 2f 20
FIXUPS: 21f70 15 1927 10 10 10 10 10 ffffff30 ffffffe0 ffffffa7 fffffff8
FIXUPS: 234da fffffff8 fffffffb fffffffa ffffffeb fffffff9 ffffffe2 ffffffc6
FIXUPS: 233b1 ffffff3b ffffff41 ffffff9b ffffffbc 586 ffffffce ffffffd7
FIXUPS: 235e1 fffffff9 fffffffb ffffffed fffffff9 ffffffde 1df4 ffffffaf
FIXUPS: 252ce ffffff4f ffffffde ffffff6f fffffff9 ffffffb1 ffffffde ffffff76
FIXUPS: 25061 49f ffffffef ffffffbf ffffff71 fffffff9 ffffeca2 ffffffc9
FIXUPS: 23eed fffffff1 ffffffef ffffffe4 ffffffba ffffffaf fffffe47 fffffe72
FIXUPS: 23857 10 d a e 10 212c fffffe4a fffffdc9 fffffffb ffffffe0 fffffffb
FIXUPS: 255ac fffffff9 ffffffe2 ffffffa0 fffff6bc ffffffec fffffff9 ffffffcb
FIXUPS: 24b54 ffffffef fffffff9 ffffffa4 fffffff9 ffffff7d fffffff9 ffffff19
FIXUPS: 24944 63b ffffff01 ffffff0e ffffffe2 ffffffd1 ffffffac ffffffaa
FIXUPS: 253df fffffff0 fffe8da8 23 6e4f ffffff76 fffffecb ffffff27 1c fffffee1
FIXUPS: 14831 88 8b 2d6 11 fffffbd7 fffffcef 217 fffffb49 35 1a 15 d 1196a
FIXUPS: 25b95 ffffff53 ffffffef ffffffdc fffffff5 fffffff4 ffffffc5 fffffff5
FIXUPS: 25a43 ffffff90 fffe9298 13 18 32 4c c 16 16 27 20 1f 13 18 35 4c
FIXUPS: ee6a 16 16 41 81 14 47 11 2d fffff631 fffffcc3 fffffd09 3e 5d 85
FIXUPS: e129 28 1f92 e 2b8 1a6 45 ffffeb36 5e 12 35 1c ab 26 5e 9b 1e fffff6d7
FIXUPS: ea96 c 16 16 27 21 13 18 23 1d 4c c 16 16 27 20 2020 1af 9b 224
FIXUPS: 11289 9b 263 1a5 9b 263 1a5 ffffeccc e9 fffffda1 fffffedc 2e 71
FIXUPS: 106d7 ffffee05 11 4d b 15 2b 1e3 89 e 239 b cb b 424 ffffdb1d 177
FIXUPS: dca0 7b 5a 12 fffff578 31 48 4e 2e 48 4e 2e 39 39 5c 17 4e 17 64d7
FIXUPS: 13d3c fffff220 fffff655 7bf fffff6a4 fffff85e 28a 52 ed 1de ffffe82f
FIXUPS: 4098 10 22 d 5e 49 8 7c 43 24 12 16 5a 43 81 1f c 29 9d 91df 25
FIXUPS: d6c4 17 21 67 4a 22 6a 62 1b 126 59 ffff5a77 22 56 22 56 27 12
FIXUPS: 35fc 12 1c 1b9 19 138 12 a4 127 b ee 6e 10 63 49 8 7c 16 52 63
FIXUPS: 3e95 16 1e be a3 ffffe37d a 2d 2a f 12 14 21 41 56 34 1c 12d 6f0
FIXUPS: 2d6f 128 150 14 d6 33 33 1a 31 1c 1c 53 2b d1 56 2b d1 28 ffffe72f
FIXUPS: 1bdb 23 2e f 31 f 1e 17 95 23 d ae d 2d 52 5d d d6 52 82 95 a6
FIXUPS: 2225 1b 33 32 12 16 23 32 4d ffffeddf 24 13 15 12 12 12 16 15 d
FIXUPS: 1214 19 28 d c 52 2e 121 14 2f 16 29 1f 98 74 d 5a 1dd d d 1c 69
FIXUPS: 6f3b 12 d 2a b0 3d 1c b1 2c0 137 73 17d fc 20 60 7f ffff96e9 f
FIXUPS: 1032 12 12 c c 16 11 11 1b 1b 1b f 12 12 4cea c7 13f 14d 62 42
FIXUPS: 6245 2e 20 16 1f 10d 4c 20 2f 1e 1e 82 3c 1b0 13d c0 13d 6d 5c
FIXUPS: 6ba2 fb 145 7a 52 24 57 ffffd888 12 25d 50 108 116 51f 41 d 43
FIXUPS: 524b 49 1d d1 3f 3e 31 5c 68 a 2a 17 2a 3d aa 1a9 34f b1 6b fc
FIXUPS: 5d70 60 2abf 3f 219 301 dd 61 49 215 175 cc 94 2b cc 2e 70 235
FIXUPS: 9856 1d1 ec 20 1f ffffa9f7 8f 11 27 17 33 bc 11 5e 12 d 3414 127
FIXUPS: 7cf0 23 2e 11 23 3a 4a e1 16 e1 16 19 14d 2a 21 27 1a 16 20 28
FIXUPS: 838e 16f 24 aa da 2a ae 40 45 40 2d2f e 6c 17 16 1c 71 d 6d 42
FIXUPS: b773 4f 72 b6 116 27 1a 5f 12 16 ffffbe71 27 1c 34 4a b9 11 23
FIXUPS: 7b11 11 23 31 2c41 77 86 1ef 1c b1 20 cd 67 d3 67 61 8e 49 19 54
FIXUPS: afb5 d 1c 71 d 2b d 4f 72 e4 58 1b 67 11a 18 72 137b 44 fa 1e 4c
FIXUPS: c9ec 99 5e 66 6b 19 2c9 24 64 188 10a ffffc9c9 114 a d 3c d 1e3
FIXUPS: 9f37 8d 1ef 1c e7 32 fd 5e 9a 160c 7d 1e 16 30 d 99 51 96 12 12d
FIXUPS: beb2 123 9e 6d 11 b4 11 15 19 54 16 51 82 14 20 c1 35 b0 d1 15
FIXUPS: c7da
